:020000040800F2
:10000000D0530020B9790008194600081B460008A3
:100010001F4600082346000827460008000000008D
:100020000000000000000000000000002B46000857
:100030002D460008000000002F4600083146000849
:10004000D3790008D3790008D3790008D379000860
:10005000D3790008D3790008D3790008D379000850
:10006000D3790008D3790008D3790008D379000840
:10007000D3790008D3790008D3790008D379000830
:10008000D3790008D3790008D3790008D379000820
:10009000D3790008D3790008D3790008D379000810
:1000A000D3790008D3790008D3790008D379000800
:1000B000D3790008D3790008D37900082F480008C5
:1000C000D3790008D3790008D3790008D3790008E0
:1000D000D3790008D3790008D3790008D3790008D0
:1000E000D3790008D3790008D3790008D3790008C0
:1000F000D3790008D3790008D3790008D3790008B0
:10010000000000000000000000000000D37900089B
:10011000D3790008D3790008D3790008D37900088F
:10012000D3790008D3790008D3790008D37900087F
:10013000D3790008D3790008000000000000000017
:10014000D3790008D3790008D379000800000000B3
:10015000000000000000000000000000000000009F
:100160000000000000000000D3790008D3790008E7
:10017000D37900080000000000000000000000002B
:1001800000000000D379000800F002F800F044F805
:100190000AA090E8000C82448344AAF10107DA45E2
:1001A00001D100F039F8AFF2090EBAE80F0013F0F0
:1001B000010F18BFFB1A43F001031847AC8500007C
:1001C000CC850000103A24BF78C878C1FAD852070D
:1001D00024BF30C830C144BF04680C6070470000C1
:1001E0000023002400250026103A28BF78C1FBD840
:1001F000520728BF30C148BF0B607047692907F01C
:100200003984752907F03684002070471FB507F040
:10021000CDFD1FBD10B510BD07F08BFD1146FFF7DA
:10022000F5FF00F06EF907F0A9FD03B4FFF7F2FF48
:1002300003BC07F0ADFD0000FE49096841F6263217
:10024000B1FBF2F1484300E000BF0100A0F1010062
:10025000FAD1704710B501465D2900DD5D21F64AEF
:100260001278062A7ED2DFE802F0EF031750B1DFE2
:1002700000203E2905DCC1F13E0202EBD273C3F33C
:100280004F00202907DBA1F1200202EBD2735B10A3
:1002900040EAC32398B2F4E000202F290CDBA1F13F
:1002A0002F0240F2A2235A434FF47A73B2FBF3F2C7
:1002B0004FF6FF7303EA82102E290BDCC1F12E02E8
:1002C00040F2A2235A434FF47A7392FBF3F20243B3
:1002D00090B20AE0A1F12F0240F2A2235A434FF458
:1002E0007A7392FBF3F2024390B22E290ADC40F2B9
:1002F000A2224A434FF47A7392FBF3F240EAC222FD
:1003000090B201E040F47840BBE0002047290CDBCC
:10031000A1F14602C2EB021202EBC202642392FB7D
:10032000F3F242EA8212024390B2472902DB40F420
:1003300078400DE02F290BDBA1F12F02C2EB021256
:1003400002EBC202642392FBF3F240EAC22290B2B3
:1003500017290BDCC1EB011202EBC202642392FBF2
:10036000F3F200E070E0024390B20DE02E290BDCC6
:10037000A1F11802C2F1160202EB0212D2006423AC
:1003800092FBF3F2024390B217291EDB46291CDCD4
:100390002E290CDCA1F11702C2EB021202EBC20201
:1003A000642392FBF3F240EA821290B20DE0A1F1D5
:1003B0002F02C2F11702C2EB021202EBC202642347
:1003C00092FBF3F240EA821290B25AE0092291FBCA
:1003D000F2F20B2A23D2DFE802F02206080A0D10FF
:1003E0001316191C1F0010201CE01F201AE04FF4E8
:1003F000826017E04FF4806014E048F2100011E0D2
:1004000048F622200EE04FF608200BE04FF6C950C8
:1004100008E04FF6F07005E04FF6FF7002E043F29F
:10042000A61000BF00BF2CE0032291FBF2F2D30222
:100430004A1C032492FBF4F243EA82128B1C93FBC6
:10044000F4F31A4390B21CE03F290ADBA1F13E020B
:100450004FF4784343EA8212A1F13E031A4390B26B
:100460000CE020290ADB4A1C4FF4784303EAC2223D
:10047000A1F12003C3F11E031A4390B240F06000C3
:1004800000BF00BF10BD01466C480068B0F57A7F20
:1004900004D2C8006A4A1060684A10606748006861
:1004A000C0EBC00001EBD000644A10601046006849
:1004B000C008634A1268C2EBC20200EBD200604A75
:1004C000106010460068C008704710B501465D4ACC
:1004D000106800EBD07201EB62025A4B1A601A6886
:1004E00002EBD2735B10584C206800EBD07403EB26
:1004F0006403554C23602046026802EBD270401022
:1005000010BD08B572B601F0E9FB01F0F5FB01F092
:100510003DFD01F07AFC01F000FD01F0E2FC4FF43A
:1005200080704FF090410885402008854FF4487056
:10053000FFF782FE4FF09040008A10F4806F01D0E8
:1005400000BFFEE74FF480704FF09041886140207B
:1005500088616420FFF770FE40204FF090410885CD
:1005600000BF4FF09040008A10F4806FF9D0032054
:1005700001F0EEFD002001F009FF42F6E060334992
:1005800008603348334908604FF4FC63752200214A
:10059000084602F08AFB4FF4FC63752200210846EE
:1005A00002F076FD4FF4FC6375221146002002F044
:1005B0007CFB4FF4FC6375220021104602F068FDBD
:1005C0004FF4FC6375227A21002002F06EFB4FF499
:1005D000FC6375227A21002002F05AFD4FF4FC637F
:1005E0007522EF21002002F060FB4FF4FC637522BE
:1005F0007A21104602F04CFD4FF400400023B02257
:100600001B21009014A003F0A0FD40F2FF70002316
:100610001A464FF48771009011A003F096FD4FF435
:100620008260002310224FF4877100900EA003F027
:100630008CFD1DE094000020250000200C0000200F
:100640001000002004000020080000203448014071
:1006500020BF02001C0000203EEFF3F1F2EE3C0050
:10066000CFE0F3E7E0000000CAEEEFE8FF00000093
:1006700046F20C3000235022F3210090FEA003F03C
:1006800064FD4FF6E07000238022D8210090FCA08A
:1006900003F05BFD4FF4806000239022EA2100907C
:1006A000FAA003F052FD4AF285200023A022CA21BD
:1006B0000090F8A003F049FD40F2FF700023D02223
:1006C000D8210090F7A003F040FD4FF48260002392
:1006D000E0224FF487710090F5A003F036FD4FF44F
:1006E000FC63412275217C2002F0DFFA4FF4FC63A9
:1006F00041227A217C2002F0D8FA4FF4FC63E522F3
:100700000521C32002F0C4FC4FF6F07302220A2137
:10071000B92002F0BDFD4FF6F07302222921B92065
:1007200002F0B6FD4FF6F07302224921B92002F023
:10073000AFFD4FF6F07302226321B92002F0A8FD4D
:100740004FF6F07000238122AB210090302003F09F
:100750008BF94FF6F0700023A022AB2100903020DF
:1007600003F082F94FF6F0700023C022AB21009015
:10077000302003F079F94FF6F0700023DA22AB2134
:100780000090302003F070F94FF6F07302228421BC
:10079000B92002F07DFD4FF6F0730222A321B920AB
:1007A00002F076FD4FF6F0730222C321B92002F069
:1007B0006FFD4FF6F0730222DD21B92002F068FDD3
:1007C0004FF6F07302222321D00102F061FD4FF6B3
:1007D000F0730F221121DC2002F067FA4FF6F0735C
:1007E0000F220A21E32002F053FC0020B2490860E6
:1007F00014E0B149098888B2FFF72CFD0446AE48E1
:100800000068C0F16C0081B223461422802002F0FF
:100810004CFAA9480068401CA7490860A64800682F
:100820005D28E6DD0020A449086014E0A24909889B
:1008300088B2FFF70FFD04469F480068C0F1E6004C
:1008400081B223461422802002F02FFA9A480068D1
:10085000401C99490860984800685D28E6DD002042
:10086000954908601FE000209449086012E00021CB
:1008700091480068C0EBC002C2EB8010904A02EBC6
:1008800040008E4A126820F812108C480068401C04
:100890008A490860894800683928E8DD8648006888
:1008A000401C85490860844800683928DBDD002049
:1008B0008449087062B601F004BA8348007810F0E9
:1008C000100F12D08048006820F010007E490860A8
:1008D0007E48007850B90846007810F0040F04D123
:1008E00001207A49087004F005F85BE27748007847
:1008F0008128FADB02204FF0904188614FF6A85022
:10090000734908804FF4FA607249088000206A49F0
:1009100008606FE070486849096830F8110010F409
:10092000006F0DD06C486449096830F91100C0F5BA
:100930008050404200B268495F4A126821F81200B4
:1009400065495D4A126831F9120000EBD0714A1016
:100950006149594B1B6831F8131002EB410109B290
:100960005D4A554B1B6822F813101046524909681E
:1009700030F9110040F2E241884205DD0846114697
:100980004D4A126821F8120053484B49096830F962
:1009900011005249884206DA4FF6DA514E48464A6B
:1009A000126820F812104C484349096830F91100C8
:1009B0004749B1F90010884206DB47483E490968BB
:1009C00030F811004249088043483B49096830F932
:1009D00011004049B1F90010884206DC3E48364912
:1009E000096830F811003B49088033480068401C12
:1009F00031490860304800683F288BDD3248006884
:100A000020F00200304908602E48007800286BD1A1
:100A10002F48B0F90000142190FBF1F0401C00EBCE
:100A20008000800000B22E4908802A48B0F90000FA
:100A300000280CDB2748B0F90000142190FBF1F0EE
:100A400000EB8000800000B22649088051E0214878
:100A50000088404200B21F4908800846B0F90000F3
:100A6000142190FBF1F0401C00EB8000800000B2EC
:100A70001C490880084638E0C7E0F0FFE43A00006F
:100A8000D2E5EFEBEEE2E8E730F000007665723099
:100A90002E340000615F626976406C6973742E7257
:100AA00075000000D8EAE0EBE03A20E0E2F2EE0068
:100AB000C2FBEAEB200000003000002034000020E0
:100AC0004801002024000020200000201400002005
:100AD0002A0000202C000020C8000020DAFDFFFFC3
:100AE000260000202800002034E00088404200B2A8
:100AF0000880FE48B0F9000040F2E241884202DD81
:100B00000846FA490880FA48B0F90000F9498842D5
:100B100003DA4FF6DA50F6490880F448B0F90000DD
:100B2000F349B1F90010884251D1F048B0F9000002
:100B3000A0F58061E23906D1ED4800881E3800B288
:100B4000EB49088043E0E94800881E3000B2E749DD
:100B500008803CE00020E849086034E0E748E649C6
:100B6000096830F91100E149B1F9001088420DDD42
:100B7000DE48B0F90000E149DF4A126821F81200AE
:100B8000DF48006840F00200DD490860DB48DA49D0
:100B9000096830F91100D649B1F9001088420DDA20
:100BA000D348B0F90010D548D34A126820F8121083
:100BB000D348006840F00200D1490860CE48006880
:100BC000401CCD490860CC4800683F28C6DDCB49B1
:100BD000B1F93600FFF779FC00B2CA49088000205D
:100BE000C549086031E0C548C349096830F91100BA
:100BF000BF49B1F90010401A4FF4BA614843BB49EC
:100C0000B1F90010BA4AB2F90020891A90FBF1F04C
:100C100081B2B948007800F007003822A2EBC0008A
:100C2000C0EBC002C2EB8010B74A02EB4002B248F0
:100C30000078C0F3C2003823A3EBC00022F81010E4
:100C4000AD480068401CAC490860AB4800683F28CC
:100C5000C9DD0020AD490870A448B0F900000A21A0
:100C600090FBF1F42246AAA1AA4806F0C5FE4FF671
:100C7000F0700023072299210090A64803F065FA3E
:100C80009A48B0F900009A49B1F90010401A0321BE
:100C900090FBF1F09549B1F90010081A0A2190FB78
:100CA000F1F422469AA19B4806F0A6FE4FF6F0709A
:100CB0000023262299210090964803F046FA8B489B
:100CC000B0F900008A49B1F90010401A032190FBE5
:100CD000F1F08749B1F9001008440A2190FBF1F4C2
:100CE00022468BA18B4806F087FE4FF6F07000235A
:100CF000462299210090874803F027FA7C48B0F9F2
:100D000000000A2190FBF1F4224681A1814806F0FF
:100D100073FE4FF6F07000236022992100907D4809
:100D200003F013FA7748B0F9000000280FDA75488D
:100D30000088404200B2734908804FF6F0700023EB
:100D40002022CF2100902D2002F08EFE08E04FF6E9
:100D5000F07000232022CF2100902B2002F084FE8F
:100D60006848B0F900000A2190FBF1F201FB12047F
:100D70006448B0F9000090FBF1F523462A4666A1CD
:100D8000644806F039FE4FF6F07000232022D82187
:100D90000090604803F0D9F95948006840F0080015
:100DA000574908605648007810F0080F7ED0544824
:100DB000006820F008005249086000204E49086091
:100DC00077E100205649086069E14B490968C1EBA9
:100DD000C102C2EB81114C4A02EB4101504A126838
:100DE00031F8122044490968C1EBC103C3EB8111FA
:100DF000454B03EB41034A490968083133F81110A8
:100E0000501800EBD071C1F34F023B490968C1EBA8
:100E1000C103C3EB81113C4B03EB4103404909681B
:100E2000091D23F8112034490968C1EBC102C2EB46
:100E30008111354A02EB4101394A126831F812201A
:100E40002D490968C1EBC103C3EB81112E4B03EBA4
:100E5000410333490968091D33F81110501800EB9C
:100E6000D071C1F34F0224490968C1EBC103C3EB40
:100E70008111254B03EB410329490968891C23F89B
:100E800011201D490968C1EBC102C2EB81111E4A44
:100E900002EB4101224A126831F812201649096812
:100EA000C1EBC103C3EB8111174B00E08EE303EBF1
:100EB00041031B490968891C33F81110501800EBD5
:100EC000D071C1F34F030C490968C1EBC102C2EBF9
:100ED00081110D4A02EB410211490968491C22F8AF
:100EE000113005490968C1EBC1021BE02600002052
:100EF00028000020DAFDFFFF30000020C80000209D
:100F0000200000202E0000204801002014000020B6
:100F100025336900A80000202532692E253169009B
:100F200034000020C2EB8111FE4A02EB4102FE496F
:100F30000968891C32F81120FC490968C1EBC1031A
:100F4000C3EB8111F74B03EB4103F7490968091D16
:100F500033F81110501800EBD071C1F34F02F34970
:100F60000968C1EBC103C3EB8111EE4B03EB4103F5
:100F7000ED490968C91C23F81120EC490968C1EB47
:100F8000C102C2EB8111E74A02EB4102E64909685E
:100F9000091D32F81120E5490968C1EBC103C3EB13
:100FA0008111E04B03EB4103DF490968083133F855
:100FB0001110501800EBD071C1F34F02DB490968E2
:100FC000C1EBC103C3EB8111D64B03EB4103D649FF
:100FD0000968891D23F81120D4490968C1EBC102B1
:100FE000C2EB8111CF4A02EB4102CF490968091DCA
:100FF00032F81120CD490968C1EBC103C3EB81115F
:10100000C84B03EB4103C8490968891D33F8111027
:10101000501800EBD071C1F34F02C4490968C1EB0D
:10102000C103C3EB8111BF4B03EB4103BE49096808
:10103000491D23F81120BD490968C1EBC102C2EB6B
:101040008111B84A02EB4102B7490968891D32F89B
:101050001120B6490968C1EBC103C3EB8111B14B43
:1010600003EB4103B0490968083133F811105018F7
:1010700000EBD071C1F34F02AC490968C1EBC10369
:10108000C3EB8111A74B03EB4103A7490968C91DB5
:1010900023F81120A44800680830A3490860A2483A
:1010A000006830287FF791AEA048006808309F495B
:1010B00008609E48006838287FF783AE00209B496F
:1010C000086060E100209849086052E1974909688A
:1010D000C1EBC102C2EB8111924A02EB4101924A7B
:1010E000126831F81220914909680831C1EBC10337
:1010F000C3EB81118B4B03EB41018B4B1B6831F828
:101100001310501800EBD071C1F34F0287490968E2
:10111000091DC1EBC103C3EB8111824B03EB4101FC
:10112000814B1B6821F8132080490968C1EBC1027B
:10113000C2EB81117B4A02EB41017B4A126831F814
:1011400012207A490968091DC1EBC103C3EB811163
:10115000744B03EB4101744B1B6831F813105018AA
:1011600000EBD071C1F34F0270490968891CC1EBD3
:10117000C103C3EB81116B4B03EB41016A4B1B684D
:1011800021F8132069490968C1EBC102C2EB811142
:10119000644A02EB4101644A126831F81220634943
:1011A0000968891CC1EBC103C3EB81115D4B03EBE3
:1011B00041015D4B1B6831F81310501800EBD071E2
:1011C000C1F34F0259490968491CC1EBC103C3EB84
:1011D0008111544B03EB4101534B1B6821F8132041
:1011E00052490968891CC1EBC102C2EB81114D4A09
:1011F00002EB41014C4A126831F812204B49096850
:10120000091DC1EBC103C3EB8111464B03EB410147
:10121000454B1B6831F81310501800EBD071C1F327
:101220004F0242490968C91CC1EBC103C3EB8111DC
:101230003C4B03EB41013C4B1B6821F813203B491D
:101240000968091DC1EBC102C2EB8111354A02EBED
:101250004101354A126831F81220344909680831D1
:10126000C1EBC103C3EB81112E4B03EB41012E4BAC
:101270001B6831F81310501800EBD071C1F34F0206
:101280002A490968891DC1EBC103C3EB8111254BB4
:1012900003EB4101244B1B6821F813202349096803
:1012A000091DC1EBC102C2EB81111E4A02EB4101D3
:1012B0001D4A126831F812201C490968891DC1EBCA
:1012C000C103C3EB8111174B03EB4101164B1B68A4
:1012D00031F81310501800EBD071C1F34F021349CD
:1012E0000968491DC1EBC103C3EB81110D4B03EB31
:1012F00041010D4B1B6821F813200C490968891D19
:10130000C1EBC102C2EB8111064A02EB4101064A60
:10131000126831F81220054909680831C1EBC10390
:1013200006E00000480100203400002030000020CA
:10133000C3EB8111FE4B03EB4101FE4B1B6831F8FF
:101340001310501800EBD071C1F34F02FA4909682D
:10135000C91DC1EBC103C3EB8111F54B03EB410187
:10136000F44B1B6821F81320F2480068401CF14937
:101370000860F048006838287FF7A8AEEE4800689B
:101380000830ED490860EC48006830287FF79AAED5
:101390000020E94908609FE00020E649086091E0EC
:1013A000E5480068C0EBC001C1EB8010E04901EBEB
:1013B0004000E049096830F81100E0490860DE4863
:1013C0000068C0EBC001C1EB8010DD4901EB4000BB
:1013D000D849096830F81100D7490968C1EBC10242
:1013E000C2EB8111D74A02EB4101D24A126831F8AF
:1013F00012100844D0490968C1EBC102C2EB811147
:10140000CB4A02EB4101CB4A126831F81210084472
:1014100081B2C9480068C0EBC002C2EB8010C44A68
:1014200002EB4000C34A126820F81210C24800685C
:10143000C0EBC001C1EB8010BD4901EB4000BD49CC
:10144000096830F81100032190FBF1F0BA490968EE
:10145000C1EBC102C2EB8111B54A02EB4101B54AB1
:10146000126821F81200B4480068C0EBC001C1EB5B
:101470008010B34901EB4000AE49096830F8111003
:10148000AD480068C0EBC002C2EB8010AD4A02EB71
:101490004000A84A126820F81210A848008881B2BB
:1014A000A5480068C0EBC002C2EB8010A44A02EB62
:1014B0004000A04A126820F812109E480068401CA4
:1014C0009C4908609B48006838287FF769AF9A48B4
:1014D0000068401C984908609748006838287FF7E2
:1014E0005BAF00209449086031E00020914908601A
:1014F00024E091490968C1EBC102C2EB81118C4A19
:1015000002EB41018B4A126831F81240E11704EBFB
:1015100011710811FEF79EFE87490968C1EBC102EF
:10152000C2EB8111824A02EB4101824A126821F822
:10153000120080480068401C7E4908607D480068B1
:101540003828D6DD7C480068401C7B4908607A4812
:1015500000683828C9DD1D20774908602CE07648EE
:101560000068C0EBC001C1EB8010714901EB400085
:10157000B0F840004FF6FF7148406F490968C1EB71
:10158000C102C2EB81116A4A02EB4101A1F840009D
:1015900002F564606849096830F811004FF6FF7180
:1015A000484002F56461644A126821F812006248FA
:1015B0000068401C604908605F4800682328CEDD51
:1015C00002F05AFE02204FF0904108855E480078F4
:1015D00010F0200F7ED05C48006820F020005A49AF
:1015E00008600846006880F001000860084600783E
:1015F00010F0020F0ED00846007810F0010F09D04D
:101600004FF4784000233822D82100904FA002F0F8
:101610009CFD08E04FF4784000233822D821009048
:101620004DA002F092FD04214FF0A04003F052FEC5
:10163000012867D14FF0A04003F04FFD41F6302163
:1016400000FB01F4E01704EB105000133A49086066
:1016500008460068FEF717FF37490860084641A1B1
:101660000268424806F0C8F943F2A610002360223F
:10167000D82100903D4802F068FD2F48006840F6F0
:101680000251884203DA00202B49086019E02A48F9
:10169000006841F26801884203DD64202649086041
:1016A0000FE025480068A0F602502349086008466C
:1016B000006800EB80004000572190FBF1F01E49CC
:1016C00008601D482AA10268284806F095F91A48C2
:1016D000006800E016E00F280ADA4FF47840002393
:1016E000602240F217110090204802F02EFD09E020
:1016F0004FF6FF700023602240F2171100901B4844
:1017000002F023FD1048008810F4807F64D00E485A
:10171000006820F480700C4908601E20164908609B
:1017200016480068A0F53851E0394ED1064827E048
:101730004801002034000020300000203800002044
:10174000AA1A00200C34002020000020C2EDE52061
:10175000F8EAE0EBFB2100002020202020202020C0
:10176000202000002534756D56000000A8000020E0
:10177000253375252500000018000020344801405D
:10178000007810F0040F10D040F2FF7000231A46CA
:101790004FF487710090FE4802F0D7FCFD480068C6
:1017A00020F00400FB4908600FE040F2FF700023C6
:1017B0001A464FF487710090F7A002F0C6FCF54876
:1017C000006840F00400F3490860F548F5490860F6
:1017D00042F6E060F4490860EE48007810F0400FEF
:1017E0007ED0EC48006820F04000EA4908601E20E6
:1017F000EE490860EC480068A0F53851E03976D130
:10180000EB480078401CEA49087008460078012837
:1018100004D0022817D003284DD130E040F2FF70E9
:101820000023C0224FF487710090E2A002F08DFCEB
:1018300040F2FF700023D0224FF487710090DFA0A8
:1018400002F083FC52E04FF4C870DE490880A0200B
:10185000DD49088040F2FF700023C0224FF48771F9
:101860000090DAA002F071FC40F2FF700023D02259
:101870004FF487710090D7A002F067FC36E04FF478
:101880004870D04908806FF03100CF490880400D82
:101890000023C0224FF487710090D0A002F055FCC5
:1018A00040F2FF700023D0224FF487710090CDA04A
:1018B00002F04BFC1AE040F2FF700023C0224FF40C
:1018C00087710090BBA002F040FC40F2FF70002343
:1018D000D0224FF487710090C4A002F036FC01E0E2
:1018E0000CE004E00020B249087000BF00BFAC4823
:1018F000AC49086042F6E060AB490860A548008842
:1019000010F4006F37D0A348006820F40060A149AC
:1019100008601E20A5490860A148A249086042F657
:10192000E060A1490860B3480078401CB1490870E4
:1019300008460078052801DD002008700020AE4927
:10194000086014E0AC49098888B2FEF783FC0446BD
:10195000A9480068C0F16C0081B22346142280209F
:1019600001F0A3F9A4480068401CA3490860A248FC
:1019700000685D28E6DD8748008810F4806F7DD020
:101980008448006820F48060824908601E208749EE
:10199000086083488349086042F6E0608249086035
:1019A0001D20954908602CE093480068C0EBC001F9
:1019B000C1EB8010914901EB4000B0F840004FF6B8
:1019C000FF7148408C490968C1EBC102C2EB81112B
:1019D0008A4A02EB4101A1F8400002F564608649A1
:1019E000096830F811004FF6FF71484002F5646154
:1019F000814A126821F812007F480068401C7E4925
:101A000008607D4800682328CEDD00207A49086000
:101A100077E000207A4908606AE0774B1B68C3EBE7
:101A2000C304C4EB8313754C04EB4303744C246868
:101A300033F81420724B1B885B007C3399B26E4BD9
:101A40001B885B009B1C98B201F043F86A4B1B6833
:101A5000C3EBC304C4EB8313684C04EB4303684C2F
:101A6000246833F81420664B1B885B007D3399B2E1
:101A7000614B1B885B009B1C98B200E009E101F000
:101A800028F85D4B1B68C3EBC304C4EB83135B4CAA
:101A900004EB43035A4C246833F81420584B1B883A
:101AA0005B007C3399B2544B1B885B00DB1C98B203
:101AB00001F00FF8504B1B68C3EBC304C4EB831356
:101AC0004E4C04EB43034E4C246833F814204C4B2B
:101AD0001B885B007D3399B2474B1B885B00DB1C86
:101AE00098B200F0F6FF46480068401C4449086080
:101AF00043480068382890DD3F480068401C3E4954
:101B000008603D480068382883DD2E48B0F90000A1
:101B10000A2190FBF1F42246AFF60C41394805F05A
:101B20006BFF4FF6F0700023812299210090354819
:101B300002F00BFB2348B0F900002349B1F9001073
:101B4000401A032190FBF1F01E49B1F90010081A68
:101B50000A2190FBF1F42246AFF64C41294805F0EA
:101B60004BFF4FF6F0700023A022992100902548EA
:101B700002F0EBFA1348B0F900001349B1F9001074
:101B8000401A032190FBF1F00F49B1F900103BE03E
:101B90006006000820000020D1F2E0F0F200000012
:101BA00020BF02001C000020344801401800002023
:101BB00024000020202020202000000020F4E8EA5B
:101BC000F1000000260000202800002020343060B2
:101BD00043000000203136604300000020383060B0
:101BE00043000000202D35604300000020E0E2F2B9
:101BF000EE000000250000203000002048010020F9
:101C000034000020A800002008440A2190FBF1F4D1
:101C10002246AFF604512C4805F0EEFE4FF6F07068
:101C20000023C02299210090274802F08EFA27480D
:101C3000B0F900000A2190FBF1F42246AFF63051D2
:101C4000214805F0D9FE4FF6F0700023DA229921E1
:101C500000901D4802F079FA00201D49086014E048
:101C60001B49098888B2FEF7F5FA0446184800684F
:101C7000C0F1E60081B223461422802001F015F85D
:101C800013480068401C12490860114800685D282C
:101C9000E6DD1048007810F0800F12D072B64020B8
:101CA0004FF0904188618000088500200A49086053
:101CB0006420FEF7C1FA40204FF09041088500BF34
:101CC000FEE7FEF7FABD0000A80000202800002073
:101CD00030000020200000203448014010B503F0FF
:101CE00061FC30B903F045FCBB2003F005FD03F0B7
:101CF0004BFC05F007FE10BD1CB50121480404F0A3
:101D000049FE0121880404F045FE4FF0904003F0A5
:101D100051FEBA4803F04EFE04220821B74803F0F2
:101D200032FF04220921B54803F02DFF4FF4407023
:101D3000009002208DF8040003208DF8050001209A
:101D40008DF806008DF807006946AC4803F099FE4F
:101D5000012207214FF0904003F015FF80200090F2
:101D600002208DF8040000208DF806008DF8070091
:101D700003208DF8050069464FF0904003F081FE86
:101D80000120009003208DF8040000208DF807004A
:101D900069464FF0904003F074FE40F2FF4000901F
:101DA00000208DF804008DF8060002208DF8070051
:101DB00003208DF805006946904803F062FE4FF459
:101DC000C060009001208DF8070069464FF09040F8
:101DD00003F057FE4FF47840009001208DF8040086
:101DE00000208DF806008DF8070003208DF805000F
:101DF0006946824803F045FE48F27E10009069462D
:101E00004FF0904003F03DFE1CBD10B58EB0002495
:101E10004FF4907004F0E7FC0121080704F0BAFDCC
:101E200006A802F012FF01214FF0A04002F0A3FF2C
:101E30000A2073490968734AB1FBF2F1484300E094
:101E400000BF0100A0F10100FAD14FF0A04002F064
:101E500071FF4FF0A04002F061FF00BF4FF0A040C3
:101E600002F070FF0028F9D14FF0A04002F05BFFB4
:101E70000446002001900290039004908DF8140015
:101E800001A94FF0A04002F00DFF4FF40050069062
:101E900000200790089009900A900B900C90012068
:101EA0008DF8340006A94FF0A04002F0B1FE0423E3
:101EB000012211464FF0A04003F040F801214FF0FD
:101EC000A04002F020FF00BF01214FF0A04003F02E
:101ED00001FA0028F8D04FF0A04003F0D3F80EB07C
:101EE00010BD00B587B00121480504F06DFD4648DE
:101EF00003F07AFE45480090002001900290039084
:101F000004900590069069463F4803F086FE012143
:101F10003D4803F0BDFE07B000BD00B589B001210A
:101F2000880404F044FD3A4804F0AEFD0020ADF80A
:101F30002000ADF81A0042F6E06007900020ADF8EE
:101F40001800ADF8220006A9314804F027FE6020F1
:101F500001900120ADF808000020ADF80A000390C0
:101F6000ADF81000ADF81400ADF81200ADF8160091
:101F700001A9274804F0BFFE0121254805F016FB02
:101F80000121234804F0ABFE09B000BD38B51F2085
:101F90008DF8000003208DF801008DF8020001206B
:101FA0008DF80300684604F01CF8154800684FF4EB
:101FB0007A72B0FBF2F1481EB0F1807F00D31BE0D3
:101FC000481E4FF0E022506150170F22002807DA18
:101FD00013071D0E0F4B00F00F04241F1D5503E0C7
:101FE00013071C0E0C4B1C5400BF00204FF0E022C6
:101FF00090610720106100BF38BD00000004004858
:102000009400002000127A00005400407A25E0007D
:102010000048014018ED00E000E400E003468B4278
:1020200001DA084670479A4201DA1046FAE7184684
:10203000F8E74FF48041FE4A1180491011804910A1
:102040001180C1B2C2434FF47F0303EA024211433D
:10205000F74A103A11604FF4804111608910116005
:102060004900116070474FF48041F14A1180891096
:102070001180C1B2C2434FF47F0303EA024211430D
:10208000EB4A103A11604FF48041116089101160E1
:1020900070474FF48041E64A103A1160E44928390C
:1020A00009686FF30F01E24A283A11604FF480513A
:1020B000DF4A11804900DE4A103A11608900DC4A8B
:1020C000118000BFDA4918390988C8B24FF40041BD
:1020D000D74A103A1160C9101160D54928390968EA
:1020E00045F255521143D24A283A1160704710B553
:1020F00004463620FFF79DFF34B1012C08D0022C96
:102100000AD0032C10D10BE04820FFF7ACFF0BE006
:102110002820FFF7A8FF07E08820FFF7A4FF03E0CF
:10212000E820FFF7A0FF00BF00BF0CB1022C07D1D1
:10213000EF20C049088040F23F10BF49088006E008
:1021400040F23F10BB490880EF20BB49088010BD1A
:1021500010B504464FF48050B54910390860C000EE
:102160004FF090410885B24910390860B0482838CE
:10217000006845F255510843AD49283908604FF4CD
:102180007F00AB49103908601420FEF755F84FF472
:1021900000404FF0904188611420FEF74DF8012077
:1021A000FFF747FF0A20FEF747F8CB20FFF741FF74
:1021B0003920FFF758FF2C20FFF755FF0020FFF7CD
:1021C00052FF3420FFF74FFF0220FFF74CFFCF20D4
:1021D000FFF72FFF0020FFF746FFC120FFF743FF67
:1021E0003020FFF740FFE820FFF723FF8520FFF7AF
:1021F0003AFF0020FFF737FF7820FFF734FFEA208F
:10220000FFF717FF0020FFF72EFF0020FFF72BFF3F
:10221000ED20FFF70EFF6420FFF725FF0320FFF7F7
:1022200022FF1220FFF71FFF8120FFF71CFFF7207E
:10223000FFF7FFFE2020FFF716FFC020FFF7F9FE93
:102240002320FFF710FFC120FFF7F3FE1020FFF758
:102250000AFFC520FFF7EDFE2B20FFF704FF2B2020
:10226000FFF701FF2046FFF742FFB120FFF7E1FE35
:102270000020FFF7F8FE1B20FFF7F5FEB620FFF762
:10228000D8FE0A20FFF7EFFE0220FFF7ECFEF22057
:10229000FFF7CFFE0220FFF7E6FE3A20FFF7C9FE68
:1022A0000520FFF7E0FE2620FFF7C3FE0120FFF721
:1022B000DAFE2120FFF7BDFEE020FFF7BAFE0F2077
:1022C000FFF7D1FE3120FFF7CEFE2B20FFF7CBFE2C
:1022D0000C20FFF7C8FE0E20FFF7C5FE0820FFF711
:1022E000C2FE4E20FFF7BFFEF120FFF7BCFE3720F5
:1022F000FFF7B9FE0720FFF7B6FE1020FFF7B3FE89
:102300000320FFF7B0FE0E20FFF7ADFE0920FFF718
:10231000AAFE0020FFF7A7FEE120FFF78AFE0020BB
:10232000FFF7A1FE0E20FFF79EFE1420FFF79BFE95
:102330000320FFF798FE1120FFF795FE0720FFF717
:1023400092FE3120FFF78FFEC120FFF78CFE482060
:10235000FFF789FE0820FFF786FE0F20FFF783FEB8
:102360000C20FFF780FE3120FFF77DFE3620FFF7BF
:102370007AFE0F20FFF777FE1120FFF75AFE0A20A2
:10238000FDF75AFF2920FFF754FE10BD2DE9F04359
:1023900007464FF0000800262648B0F800902A2093
:1023A000FFF747FE00BF4FF48050214908808000AE
:1023B0000880F043000A4FF47F0101EA004040EA40
:1023C00016201B49103908604FF4804008601849F6
:1023D0000880F0434FF47F0101EA00403043144984
:1023E000103908604FF4804008608010086000BF1A
:1023F00000BF0F490880800008806FEA0900000ACA
:102400004FF47F0101EA004040EA192008491039E1
:1024100008604FF4804008600549088009F0FF001B
:102420006FEA09014FF47F0202EA0141084305E027
:10243000280400484000002042000020FE491039D6
:1024400008604FF4804008608010086000BF00BF43
:10245000FA48B0F800902B20FFF7EBFD00BF4FF4D7
:102460008050F549088080000880F043000A4FF44E
:102470007F0101EA004040EA1620EF491039086068
:102480004FF480400860EC490880F0434FF47F012E
:1024900001EA00403043E849103908604FF48040B9
:1024A00008608010086000BF00BFE349088080001A
:1024B00008806FEA0900000A4FF47F0101EA00403A
:1024C00040EA1920DC49103908604FF48040086068
:1024D000D949088009F0FF006FEA09014FF47F0233
:1024E00002EA01410843D449103908604FF48040A2
:1024F00008608010086000BF00BF2C20FFF799FD26
:102500004FF40050CC49103908604010CA49088087
:102510003C12FDB200BFAAE14FF48040C6490880DA
:10252000E0B2E1434FF47F0202EA01410843C249AD
:10253000103908604FF480400860BF490880E8B255
:10254000E94302EA01410843BB49103908604FF4EE
:1025500080400860B8490880E0B2E14302EA0141E6
:102560000843B549103908604FF480400860B2490B
:102570000880E8B2E94302EA01410843AE49103954
:1025800008604FF480400860AB490880E0B2E14346
:1025900002EA01410843A849103908604FF480401D
:1025A0000860A5490880E8B2E94302EA014108430E
:1025B000A149103908604FF4804008609E490880A6
:1025C000E0B2E14302EA014108439B491039086047
:1025D0004FF48040086098490880E8B2E94302EA75
:1025E000014108439449103908604FF48040086065
:1025F00091490880E0B2E14302EA014108438E4973
:10260000103908604FF4804008608B490880E8B2B8
:10261000E94302EA014108438749103908604FF451
:102620008040086084490880E0B2E14302EA014149
:1026300008438149103908604FF4804008607E49A2
:102640000880E8B2E94302EA014108437A491039B7
:1026500008604FF48040086077490880E0B2E143A9
:1026600002EA014108437449103908604FF4804080
:10267000086071490880E8B2E94302EA0141084371
:102680006D49103908604FF4804008606A4908803D
:10269000E0B2E14302EA01410843674910390860AA
:1026A0004FF48040086064490880E8B2E94302EAD8
:1026B000014108436049103908604FF480400860C8
:1026C0005D490880E0B2E14302EA014108435A490A
:1026D000103908604FF48040086057490880E8B21C
:1026E000E94302EA014108435349103908604FF4B5
:1026F0008040086050490880E0B2E14302EA0141AD
:1027000008434D49103908604FF4804008604A4939
:102710000880E8B2E94302EA01410843464910391A
:1027200008604FF48040086043490880E0B2E1430C
:1027300002EA014108434049103908604FF48040E3
:1027400008603D490880E8B2E94302EA01410843D4
:102750003949103908604FF48040086036490880D4
:10276000E0B2E14302EA014108433349103908600D
:102770004FF48040086030490880E8B2E94302EA3B
:10278000014108432C49103908604FF4804008602B
:1027900029490880E0B2E14302EA014108432649A1
:1027A000103908604FF48040086023490880E8B27F
:1027B000E94302EA014108431F49103908604FF418
:1027C000804008601C490880E0B2E14302EA014110
:1027D00008431949103908604FF4804008601649D1
:1027E0000880E8B2E94302EA01410843124910397E
:1027F00008604FF4804008600F490880E0B2E14370
:1028000002EA014108430C49103908604FF4804046
:10281000086009490880E8B2E94302EA0141084337
:102820000549103908604FF480400860024908806B
:10283000E0B2E14304E00000280400484200002028
:1028400002EA01410843FE4908604FF480400860F5
:10285000FB4910310880E8B2E94302EA014108432C
:10286000F74908604FF48040086008F10108B8F5A6
:10287000965FFFF451AE4FF48050F1490860BDE817
:10288000F0832DE9F04F07460C4615461E46A74239
:1028900002DD67407C406740B54202DD75406E4016
:1028A0007540E848028800213846FFF7B7FB074625
:1028B000E448028800212046FFF7B0FB0446E248C6
:1028C000028800212846FFF7A9FB0546DE4802885A
:1028D00000213046FFF7A2FB0646E01B401CDB4907
:1028E0000860701B401C09684843D8490860B84616
:1028F000A1462A20FFF79DFB00BF4FF48050D0492E
:1029000010310880800008806FEA0800000A4FF448
:102910007F0101EA004040EA1820C94908604FF4ED
:1029200080400860C6491031088008F0FF006FEA57
:1029300008014FF47F0202EA01410843C0490860E0
:102940004FF4804008608010086000BF00BFBC49A1
:1029500010310880800008806FEA0900000A1146E3
:1029600001EA004040EA1920B54908604FF4804070
:102970000860B3491031088009F0FF006FEA0901CF
:1029800002EA01410843AE4908604FF48040086004
:102990008010086000BF00BFA846B1462B20FFF79B
:1029A00048FB00BF4FF48050A549103108808000DB
:1029B00008806FEA0800000A4FF47F0101EA004036
:1029C00040EA18209E4908604FF4804008609C4906
:1029D0001031088008F0FF006FEA08014FF47F0211
:1029E00002EA01410843964908604FF480400860BC
:1029F0008010086000BF00BF91491031088080003E
:102A000008806FEA0900000A114601EA004040EA26
:102A100019208B4908604FF48040086088491031C4
:102A2000088009F0FF006FEA090102EA014108434A
:102A3000834908604FF4804008608010086000BF40
:102A400000BF2C20FFF7F5FA4FF400507C490860D6
:102A500040107B491031088009984FEA202A0998D4
:102A600000F0FF0B00207A49086026E04FF4804018
:102A70007349103108800AF0FF006FEA0A014FF431
:102A80007F0202EA014108436D4908604FF480402B
:102A900008606B49103108800BF0FF006FEA0B01F2
:102AA00002EA01410843664908604FF4804008602B
:102AB00067480068401C66490860654800686349CB
:102AC00009688842D2D34FF480505D490860BDE860
:102AD000F08F70B504460D46164600BF00BF2A2091
:102AE000FFF7A7FA00BF4FF4805055491031088016
:102AF00080000880E043000A4FF47F0101EA0040B3
:102B000040EA14204E4908604FF4804008604C4968
:102B100010310880E0B2E1434FF47F0202EA014144
:102B20000843474908604FF48040086080100860FF
:102B300000BF00BF42491031088080000880E04398
:102B4000000A114601EA004040EA14203C490860AE
:102B50004FF4804008603A4910310880E0B2E14308
:102B600002EA01410843364908604FF4804008609A
:102B70008010086000BF00BF00BF2B20FFF759FA8C
:102B800000BF4FF480502E4910310880800008802B
:102B9000E843000A4FF47F0101EA004040EA1520B3
:102BA000274908604FF480400860254910310880AB
:102BB000E8B2E9434FF47F0202EA014108432049A9
:102BC00008604FF4804008608010086000BF00BFBC
:102BD0001B491031088080000880E843000A114634
:102BE00001EA004040EA1520154908604FF4804092
:102BF0000860134910310880E8B2E94302EA014154
:102C000008430F4908604FF4804008608010086056
:102C100000BF00BF2C20FFF70CFA00BF00BF4FF42D
:102C2000805007491031088080000880F043000A76
:102C30004FF47F0101EA004040EA1620004909E014
:102C400018040048400000204200002048000020F6
:102C50004C00002008604FF480400860FE49088066
:102C6000F0B2F1434FF47F0202EA01410843FA490E
:102C7000103908604FF4804008608010086000BF81
:102C800070BD2DE9F84105460C4616461F46DDF895
:102C90001C80E01983B2A81981B222462846CDF8DB
:102CA0000080FFF7EEFDBDE8F8812DE9F043054611
:102CB0000C4617461E46E8191FFA80F92A20FFF72E
:102CC000B8F900BF4FF48050E349088080000880C5
:102CD000E843000A4FF47F0101EA004040EA152072
:102CE000DD49103908604FF480400860DA490880F7
:102CF000E8B2E9434FF47F0202EA01410843D649B2
:102D0000103908604FF4804008608010086000BFF0
:102D100000BFD1490880800008806FEA0900000ADE
:102D2000114601EA004040EA1920CB4910390860F9
:102D30004FF480400860C849088009F0FF006FEA3E
:102D4000090102EA01410843C349103908604FF400
:102D5000804008608010086000BF00BF00BF2B20CB
:102D6000FFF767F900BF4FF48050BB49088080002F
:102D70000880E043000A4FF47F0101EA004040EA86
:102D80001420B549103908604FF480400860B249FA
:102D90000880E0B2E1434FF47F0202EA01410843B8
:102DA000AD49103908604FF4804008608010086019
:102DB00000BF00BFA849088080000880E043000AE7
:102DC000114601EA004040EA1420A3491039086086
:102DD0004FF480400860A0490880E0B2E14302EA75
:102DE000014108439C49103908604FF48040086055
:102DF0008010086000BF00BF2C20FFF71AF94FF0C9
:102E000000082AE000BF4FF48050934908808000FA
:102E10000880F043000A4FF47F0101EA004040EAD5
:102E200016208D49103908604FF4804008608A49A7
:102E30000880F0B2F1434FF47F0202EA01410843F7
:102E40008549103908604FF48040086080100860A0
:102E500000BF08F101001FFA80F8B845D2DBBDE8D9
:102E6000F0832DE9F04F85B004460D4690469A4612
:102E70000E9EA8EB04000490AAEB050003900498B2
:102E8000002801DB014600E041428B46444501DA5F
:102E9000012001E04FF0FF3002900398002801DB91
:102EA000014600E041424F42554501DA012001E070
:102EB0004FF0FF3001900BEB070900BF00BF00BFD0
:102EC00000BF2A20FFF7B5F800BF4FF480506249D9
:102ED000088080000880E043000A4FF47F0101EA87
:102EE000004040EA14205C49103908604FF48040EB
:102EF000086059490880E0B2E1434FF47F0202EADA
:102F0000014108435449103908604FF4804008607B
:102F10008010086000BF00BF4F4908808000088013
:102F2000E043000A114601EA004040EA14204A4901
:102F3000103908604FF48040086047490880E0B2CB
:102F4000E14302EA014108434349103908604FF464
:102F5000804008608010086000BF00BF00BF2B20C9
:102F6000FFF767F800BF4FF480503B4908808000AE
:102F70000880E843000A4FF47F0101EA004040EA7C
:102F800015203549103908604FF4804008603249F7
:102F90000880E8B2E9434FF47F0202EA01410843A6
:102FA0002D49103908604FF4804008608010086097
:102FB00000BF00BF2849088080000880E843000A5D
:102FC000114601EA004040EA152023491039086003
:102FD0004FF48040086020490880E8B2E94302EAE3
:102FE000014108431C49103908604FF480400860D3
:102FF0008010086000BF00BF2C20FFF71AF800BF48
:1030000000BF4FF480501449088080000880F043CE
:10301000000A4FF47F0101EA004040EA16200E4901
:10302000103908604FF4804008600B490880F0B206
:10303000F1434FF47F0202EA014108430649103987
:1030400008604FF4804008608010086000BF00BF37
:103050004FEA4900009001E0280400480098B84277
:1030600006DB444500D10FE0B9440298204484B205
:10307000009858453FF722AF554500D104E0D944A8
:103080000198284485B219E700BF05B0BDE8F08F6C
:103090002DE9F04304460D4617461E4600BF2A2080
:1030A000FEF7C7FF00BF4FF48050FE490880800044
:1030B0000880E043000A4FF47F0101EA004040EA43
:1030C0001420F849103908604FF480400860F54931
:1030D0000880E0B2E1434FF47F0202EA0141084375
:1030E000F049103908604FF4804008608010086093
:1030F00000BF00BFEB49088080000880E043000A61
:10310000114601EA004040EA1420E64910390860FF
:103110004FF480400860E3490880E0B2E14302EAEE
:1031200001410843DF49103908604FF480400860CE
:103130008010086000BF00BFE8191FFA80F92B203B
:10314000FEF777FF00BF4FF48050D649088080001B
:103150000880E843000A4FF47F0101EA004040EA9A
:103160001520D049103908604FF480400860CD49DF
:103170000880E8B2E9434FF47F0202EA01410843C4
:10318000C849103908604FF480400860801008601A
:1031900000BF00BFC3490880800008806FEA0900B3
:1031A000000A114601EA004040EA1920BD491039E1
:1031B00008604FF480400860BA49088009F0FF00B9
:1031C0006FEA090102EA01410843B6491039086073
:1031D0004FF4804008608010086000BF00BF2C20C2
:1031E000FEF727FF4FF000082AE000BF4FF48050A1
:1031F000AC49088080000880F043000A4FF47F014A
:1032000001EA004040EA1620A649103908604FF450
:1032100080400860A3490880F0B2F1434FF47F0278
:1032200002EA014108439F49103908604FF4804089
:1032300008608010086000BF08F101001FFA80F8E4
:10324000B845D2DBBDE8F0832DE9F04105460E46D6
:1032500017461C46DDF8188043463A463146284654
:10326000FFF723FD301981B243463A462846FFF75F
:103270001CFD4346224631462846FFF709FFE9195F
:1032800088B2434622463146FFF702FFBDE8F0818F
:103290002DE9FF4F81B081468A461C46039847427C
:1032A0004FF0000803984000C0F1020B00BFA9EBEB
:1032B000070086B20AEB080085B200BF00BF2A20D3
:1032C000FEF7B7FE00BF4FF48050764908808000BB
:1032D0000880F043000A4FF47F0101EA004040EA11
:1032E00016207049103908604FF4804008606D491D
:1032F0000880F0B2F1434FF47F0202EA0141084333
:103300006849103908604FF48040086080100860F8
:1033100000BF00BF6349088080000880F043000AB6
:10332000114601EA004040EA16205E491039086063
:103330004FF4804008605B490880F0B2F14302EA34
:10334000014108435749103908604FF48040086034
:103350008010086000BF00BF00BF2B20FEF769FE91
:1033600000BF4FF480504F49088080000880E84338
:10337000000A4FF47F0101EA004040EA1520494964
:10338000103908604FF48040086046490880E8B270
:10339000E9434FF47F0202EA0141084341491039F1
:1033A00008604FF4804008608010086000BF00BFD4
:1033B0003C49088080000880E843000A114601EA81
:1033C000004040EA15203749103908604FF480402A
:1033D000086034490880E8B2E94302EA0141084341
:1033E0003049103908604FF4804008608010086050
:1033F00000BF00BF2C20FEF71CFE00BF00BF4FF433
:1034000080502849088080000880E043000A4FF47B
:103410007F0101EA004040EA142022491039086087
:103420004FF4804008601F490880E0B2E1434FF448
:103430007F0202EA014108431A49103908604FF43B
:10344000804008608010086000BF00BF09EB0700E3
:1034500085B20AEB080086B200BF00BF2A20FEF743
:10346000E8FD00BF4FF480500E49088080000880BE
:10347000E843000A4FF47F0101EA004040EA1520CA
:103480000849103908604FF48040086005490880F9
:10349000E8B2E9434FF47F0202EA014108430149DF
:1034A000103901E02804004808604FF480400860AB
:1034B0008010086000BF00BFFE49088080000880BF
:1034C000E843000A114601EA004040EA1520F949A4
:1034D000103908604FF480400860F6490880E8B26F
:1034E000E94302EA01410843F249103908604FF408
:1034F000804008608010086000BF00BF00BF2B2024
:10350000FEF797FD00BF4FF48050EA490880800025
:103510000880F043000A4FF47F0101EA004040EACE
:103520001620E449103908604FF480400860E149F2
:103530000880F0B2F1434FF47F0202EA01410843F0
:10354000DC49103908604FF4804008608010086042
:1035500000BF00BFD749088080000880F043000A00
:10356000114601EA004040EA1620D24910390860AD
:103570004FF480400860CF490880F0B2F14302EA7E
:1035800001410843CB49103908604FF4804008607E
:103590008010086000BF00BF2C20FEF74AFD00BF6E
:1035A00000BF4FF48050C349088080000880E0438A
:1035B000000A4FF47F0101EA004040EA1420BD49AF
:1035C000103908604FF480400860BA490880E0B2C2
:1035D000E1434FF47F0202EA01410843B549103943
:1035E00008604FF4804008608010086000BF00BF92
:1035F00009EB070085B2AAEB080086B200BF00BF46
:103600002A20FEF716FD00BF4FF48050A94908801C
:1036100080000880E843000A4FF47F0101EA00407F
:1036200040EA1520A349103908604FF48040086033
:10363000A0490880E8B2E9434FF47F0202EA014161
:1036400008439C49103908604FF48040086080109E
:10365000086000BF00BF9749088080000880E843E9
:10366000000A114601EA004040EA1520914910394C
:1036700008604FF4804008608E490880E8B2E94352
:1036800002EA014108438B49103908604FF4804039
:1036900008608010086000BF00BF00BF2B20FEF74D
:1036A000C8FC00BF4FF48050824908808000088029
:1036B000F043000A4FF47F0101EA004040EA16207F
:1036C0007C49103908604FF48040086079490880CF
:1036D000F0B2F1434FF47F0202EA01410843754919
:1036E000103908604FF4804008608010086000BF07
:1036F00000BF7049088080000880F043000A11462E
:1037000001EA004040EA16206A49103908604FF487
:103710008040086067490880F0B2F14302EA014145
:1037200008436449103908604FF4804008608010F5
:10373000086000BF00BF2C20FEF77BFC00BF00BF6D
:103740004FF480505B49088080000880E043000A05
:103750004FF47F0101EA004040EA14205549103936
:1037600008604FF48040086052490880E0B2E143AD
:103770004FF47F0202EA014108434E4910390860C4
:103780004FF4804008608010086000BF00BFA9EBC4
:10379000070085B2AAEB080086B200BF00BF2A204E
:1037A000FEF747FC00BF4FF480504249088080007C
:1037B0000880E843000A4FF47F0101EA004040EA34
:1037C00015203C49103908604FF4804008603949A1
:1037D0000880E8B2E9434FF47F0202EA014108435E
:1037E0003449103908604FF4804008608010086048
:1037F00000BF00BF2F49088080000880E843000A0E
:10380000114601EA004040EA15202A4910390860B3
:103810004FF48040086027490880E8B2E94302EA93
:10382000014108432349103908604FF48040086083
:103830008010086000BF00BF00BF2B20FEF7F9FB1F
:1038400000BF4FF480501B49088080000880F0437F
:10385000000A4FF47F0101EA004040EA16201549B2
:10386000103908604FF48040086012490880F0B2B7
:10387000F1434FF47F0202EA014108430D49103938
:1038800008604FF4804008608010086000BF00BFEF
:103890000849088080000880F043000A114601EAC8
:1038A000004040EA16200349103908604FF4804078
:1038B000086001E028040048F8490880F0B2F143AC
:1038C00002EA01410843F549103908604FF480408D
:1038D00008608010086000BF00BF2C20FEF7A9FB25
:1038E00000BF00BF4FF48050EC4908808000088082
:1038F000E043000A4FF47F0101EA004040EA14204F
:10390000E649103908604FF480400860E3490880B8
:10391000E0B2E1434FF47F0202EA01410843DF498C
:10392000103908604FF4804008608010086000BFC4
:1039300000BFCDF800B0DDF800B0C3450EDC08F1E3
:1039400001008046012101EB4000834417EB080F82
:1039500004D10098B84201DC002000900098B842E1
:1039600005DD781C0746012101EB40008344002F50
:103970007FF79DAC05B0BDE8F08F2DE9F04F07460D
:10398000884691469B46C9F1000400254FEA49004C
:10399000C0F1020600BF6B041A0CA8EB050399B234
:1039A0003B1B98B25B46FFF773FB6B041A0CA8EB4A
:1039B000050399B23B1998B25B46FFF769FBB24623
:1039C000AA450BDC681C0546012101EB40000644BA
:1039D000EC4203D1A24501DC4FF0000AA24505DD0F
:1039E000601C0446012101EB40000644002CD2DD9E
:1039F000BDE8F08F2DE9F04306460D4614461F46FC
:103A0000DDF81C904FF001080FB9BDE8F083002FDE
:103A100013DD0FE04B46424629463046FFF745F995
:103A2000701E86B2681C85B208F102001FFA80F889
:103A3000601E84B2002CEDD114E0281985B20FE08D
:103A40004B46424629463046FFF72FF9701E86B294
:103A5000681E85B208F102001FFA80F8601E84B269
:103A6000002CEDD100BFD0E72DE9FF4F82B0824698
:103A70009846DDF83C9000200190BAF1200F01DA61
:103A80004FF01F0A8648007800287DD100241AE2F2
:103A9000BAF1200F0ADBBAF17F0F07DCAAF1200090
:103AA000804901EB0010005D019009E0BAF1C00F00
:103AB00006DBAAF165007B4901EB0010005D019077
:103AC0002046E11704EB5171C1F3C7054FF0000B1D
:103AD000F4E1019840FA0BF010F0010F7DD0B8F13D
:103AE000000F7BD103982044A0EBC50087B2049857
:103AF000584400EBC50086B200BF00BF2A20FEF785
:103B000098FA00BF4FF48050644908808000088014
:103B1000F843000A4FF47F0101EA004040EA172011
:103B20005E49103908604FF4804008605B490880A6
:103B3000F8B2F9434FF47F0202EA014108435749C2
:103B4000103908604FF4804008608010086000BFA2
:103B500000BF5249088080000880F843000A1146DF
:103B600001EA004040EA17204C49103908604FF440
:103B70008040086049490880F8B2F94302EA0141EF
:103B800008434649103900E0AFE108604FF4804037
:103B900008608010086000BF00BF00BF2B20FEF748
:103BA00048FA00BF4FF480503C49088080000880EC
:103BB000F043000A4FF47F0101EA004040EA16207A
:103BC0003649103908604FF4804008603349088056
:103BD000F0B2F1434FF47F0201E07AE064E002EAE0
:103BE000014108432D49103908604FF480400860B6
:103BF0008010086000BF00BF28490880800008804E
:103C0000F043000A114601EA004040EA1620234929
:103C1000103908604FF48040086020490880F0B2F5
:103C2000F14302EA014108431C49103908604FF48E
:103C3000804008608010086000BF00BF2C20FEF7A5
:103C4000F8F900BF00BF4FF480501449088080008D
:103C500008806FEA0900000A4FF47F0101EA004082
:103C600040EA19200D49103908604FF4804008607F
:103C70000A49088009F0FF006FEA09014FF47F024A
:103C800002EA014108430549103908604FF48040B9
:103C900008608010086000BF00BF0BE128040048E6
:103CA00046000020B67D0008CDF80090049A0BFB7A
:103CB0000822EB0003FB082291B2039A04FB0822BE
:103CC000EB0003FB182290B243464246FEF7D9FFB1
:103CD000F0E0B8F1000F7DD103982044A0EBC500BF
:103CE00086B20498584400EBC50087B2FE480088AD
:103CF000009000BF00BF2A20FEF79BF900BF4FF4E1
:103D00008050FA49088080000880F043000A4FF490
:103D10007F0101EA004040EA1620F44910390860AA
:103D20004FF480400860F1490880F0B2F1434FF44D
:103D30007F0202EA01410843EC49103908604FF460
:103D4000804008608010086000BF00BFE74908801D
:103D500080000880F043000A114601EA004040EA72
:103D60001620E249103908604FF480400860DF49AE
:103D70000880F0B2F14302EA01410843DB491039FF
:103D800008604FF4804008608010086000BF00BFEA
:103D900000BF2B20FEF74DF900BF4FF48050D349F0
:103DA000088080000880F843000A4FF47F0101EA90
:103DB000004040EA1720CD49103908604FF4804098
:103DC0000860CA490880F8B2F9434FF47F0202EA5A
:103DD000014100E059E00843C449103908604FF43C
:103DE000804008608010086000BF00BFBF490880A5
:103DF00080000880F843000A114601EA004040EACA
:103E00001720BA49103908604FF480400860B7495C
:103E10000880F8B2F94302EA01410843B349103976
:103E200008604FF4804008608010086000BF00BF49
:103E30002C20FEF7FEF800BF00984FF48051AB4AEB
:103E4000118089001180C143090A4FF47F0202EA00
:103E5000014141EA1021A54A103A11604FF4804116
:103E60001160A24A1180C1B2C2434FF47F0303EA3A
:103E7000024211439D4A103A11604FF48041116093
:103E80008910116000BF00BF14E0974800880090BF
:103E9000049A0BFB0822EB0003FB082291B2039A61
:103EA00004FB0822EB0003FB182290B24346424673
:103EB000FEF7E7FE0BF1010000F0FF0BBBF1080F6E
:103EC000FFF607AE641C102CFFF6E2ADB8F1000F50
:103ED0000AD18548008800900399083188B21023E0
:103EE00001220499FEF7CDFE2CE1002427E1BAF16E
:103EF000200F0ADBBAF17F0F07DCAAF120007C4912
:103F000001EB0010005D019009E0BAF1C00F06DB83
:103F1000AAF16500764901EB0010005D0190204692
:103F2000E11704EB5171C1F3C7054FF0000B01E13C
:103F3000019840FA0BF010F0010F7DD0B8F1000F9E
:103F40007BD103982044A0EBC50086B20498584466
:103F500000EBC50087B200BF00BF2A20FEF769F85A
:103F600000BF4FF480506149088080000880F04312
:103F7000000A4FF47F0101EA004040EA16205B4945
:103F8000103908604FF48040086058490880F0B24A
:103F9000F1434FF47F0202EA0141084353491039CB
:103FA00008604FF4804008608010086000BF00BFC8
:103FB0004E49088080000880F043000A114601EA5B
:103FC000004040EA16204949103908604FF480400B
:103FD000086046490880F0B2F14302EA0141084313
:103FE0004249103908604FF4804008608010086032
:103FF00000BF00BF00BF2B20FEF71BF800BF4FF42F
:1040000080503A49088080000880F843000A4FF445
:104010007F0101EA004040EA172034491039086066
:104020004FF48040086031490880F8B2F9434FF4FA
:104030007F0202EA014101E078E063E008432B4996
:10404000103908604FF4804008608010086000BF9D
:1040500000BF2649088080000880F843000A114606
:1040600001EA004040EA17202049103908604FF467
:10407000804008601D490880F8B2F94302EA014116
:1040800008431A49103908604FF4804008608010D6
:10409000086000BF00BF2C20FDF7CBFF00BF00BFB2
:1040A0004FF4805011490880800008806FEA0900B1
:1040B000000A4FF47F0101EA004040EA19200B4951
:1040C000103908604FF4804008600849088009F002
:1040D000FF006FEA09014FF47F0202EA0141084341
:1040E00002491039086005E0440000202804004817
:1040F000B67D00084FF4804008608010086000BF63
:1041000000BF13E0CDF80090049A0BFB0822EB00EF
:1041100003FB082291B2039A04FB0822EB0003FB85
:10412000182290B243464246FEF7ABFD0BF1010068
:1041300000F0FF0BBBF1080FFFF6FAAE641C102C69
:10414000FFF6D5AE06B0BDE8F08F2DE9F841044684
:104150000D4617461E46DDF81C801DE005F10900DE
:10416000FE490988884204DD0125102000FB067005
:1041700087B2CDF80080207833463A462946FFF7CB
:1041800073FC002E04DD092000FB065085B202E01E
:1041900005F1090085B2641C20780028DED1BDE855
:1041A000F8812DE9FE4F0446894690469A46DDF88F
:1041B00034B000BF002000EB0910029002981030CC
:1041C00080B201900AEBCA06E4480088401C86428F
:1041D00002D9E2480088461CBBF1010F0DD14046D0
:1041E00003F00BFD00EBC000301A400805B228199F
:1041F00005B2A5420FD225B20DE0BBF1000F01D1EF
:1042000025B208E0404603F0F8FC00EBC000301A8D
:1042100005B2281905B2D2480088A9B20090A0B210
:10422000DDE90132FEF72DFB00270CE00C98A9B266
:10423000009018F807000023029AFFF715FC05F11B
:10424000090005B27F1C18F8070030B1574504D2A9
:10425000C24800880938A842E8DCA019A84209D958
:10426000BF480088A21991B20090A8B2DDE90132DE
:10427000FEF707FBBDE8FE8FF0B5022673272A2064
:10428000FDF7D7FE00BFF002B64908808000088025
:10429000F043000A4FF47F0101EA004040EA162093
:1042A000B0491039086070030860AE490880F043D7
:1042B0004FF47F0101EA00403043AA4910390860F9
:1042C000700308608010086000BF00BFA549088027
:1042D00080000880F843000A4FF47F0101EA0040A3
:1042E00040EA17209F4910390860700308609D4913
:1042F0000880F8434FF47F0101EA004038439949B0
:1043000010390860700308608010086000BF00BFAB
:10431000022773262B20FDF78CFE00BFF80291497F
:10432000088080000880F843000A4FF47F0101EA0A
:10433000004040EA17208B49103908607803086074
:1043400088490880F8434FF47F0101EA0040384370
:10435000844910390860780308608010086000BF45
:1043600000BF8049088080000880F043000A4FF4B5
:104370007F0101EA004040EA16207A4910390860BE
:104380007803086077490880F0434FF47F0101EA21
:10439000004030437349103908607803086080108A
:1043A000086000BF00BF2C20FDF743FE38036D49B5
:1043B0001039086040106B49088000251EE1002478
:1043C00084E04FF4804067490880C4EBC400C0EB30
:1043D0008410654901EB400030F81500C043000A25
:1043E0004FF47F0101EA0040C4EBC401C1EB84112A
:1043F0005D4A02EB410131F8151040EA112059499C
:10440000103908604FF48040086056490880C4EBBA
:10441000C400C0EB8410114601EB400010F81500F9
:10442000C4EBC401C1EB841102EB410131F815105A
:10443000C9434FF47F0202EA014108434949103958
:1044400008604FF48040086046490880C4EBC4000F
:10445000C0EB8410444901EB400030F81500C04324
:10446000000A114601EA0040C4EBC401C1EB84110B
:104470003D4A02EB410131F8151040EA112039495B
:10448000103908604FF48040086036490880C4EB5A
:10449000C400C0EB8410114601EB400010F8150079
:1044A000C4EBC401C1EB841102EB410131F81510DA
:1044B000C9434FF47F0202EA0141084329491039F8
:1044C00008604FF480400860601CC4B2382C7FF74D
:1044D00078AF00248DE04FF4804022490880C4EB7F
:1044E000C400C0EB8410204901EB400030F81500F7
:1044F000C043000A4FF47F0101EA0040C4EBC4014D
:10450000C1EB8411184A02EB410131F8151040EA61
:1045100011201449103908604FF480400860114997
:104520000880C4EBC400C0EB8410114601EB4000CE
:1045300010F81500C4EBC401C1EB841102EB41017A
:1045400031F81510C9434FF47F0202EA01410843D4
:104550000449103908604FF4804007E04000002013
:104560004400002028040048480100200860284931
:104570000880C4EBC400C0EB8410264901EB400066
:1045800030F81500C043000A114601EA0040C4EBB0
:10459000C401C1EB84111F4A02EB410131F815102F
:1045A00040EA11201A49103908604FF48040086031
:1045B00017490880C4EBC400C0EB8410114601EB1E
:1045C000400010F81500C4EBC401C1EB841102EBEC
:1045D000410131F81510C9434FF47F0202EA01414D
:1045E00008430B49103908604FF480400860601C94
:1045F000C4B2382C7FF76FAF681CC5B2382D7FF777
:10460000DEAE4FF48050024910390860F0BD000062
:104610002804004848010020704700BFFEE700BFA3
:10462000FEE700BFFEE700BFFEE770477047704738
:104630004FF09040008A10F4806F16D1A1480068B6
:1046400041F28831884204D29E480068401C9D494E
:1046500008609C480068B0F5617F18D19A480068EE
:1046600040F080009849086011E0964800681928D9
:104670000AD994480068B0F5617F05D29248006875
:1046800040F040009049086000208E4908604FF0DB
:104690009040008A10F4007F16D18C48006841F2E7
:1046A0008831884204D289480068401C87490860E4
:1046B00086480068B0F5617F18D18348006840F4EF
:1046C00080608149086011E08048006819280AD993
:1046D0007E480068B0F5617F05D27B48006840F4F1
:1046E0008070794908600020784908604FF0904058
:1046F000008A10F4806F21D14FF09040008A10F4AE
:10470000007F1BD17248006841F28831884204D290
:104710006F480068401C6E4908606D480068B0F53D
:10472000617F05D16848006840F400606649086010
:104730000020644908606549086025E06448006815
:1047400010B300205F490860604908604FF0904056
:10475000008A10F4806F17D04FF09040008A10F458
:10476000007F11D05A48006819280AD958480068B3
:10477000B0F5617F05D25448006840F4007052499A
:10478000086000205249086052480068401C5149A6
:10479000086008460068642808D34B48006840F069
:1047A00010004949086000204A4908604A480068EA
:1047B000401C4949086008460068B0F5967F08D358
:1047C0004148006840F020003F490860002042490D
:1047D00008604248006888B140480068012804D158
:1047E00040204FF09041088503E040204FF0904179
:1047F00088613A480068401E3849086038480068B7
:1048000060B137480068012803D140F6B830354917
:10481000086033480068401E314908604FF09040FE
:10482000808A80F004004FF090418882704710B574
:1048300004212D4801F0A6FB002841D02B48007828
:1048400010F0010F0CD0284801F082FB27490978AD
:104850004C1E04EBD4714910254A22F8110016E0D1
:10486000214801F075FB214909784C1E04EBD471F5
:1048700049101F4A32F8111041EA002001B21B48CA
:104880000078441E04EBD470401022F81010174832
:104890000078401C154908700846007881280FDB15
:1048A00000BF2021104801F060FB0028F9D0202132
:1048B0000D4801F065FB002204210B4801F0FDF9D1
:1048C00010BD000058000020200000205C000020E7
:1048D000600000205000002054000020180000203C
:1048E0001C00002034480140005400401400002007
:1048F000C800002008B500BF4FF40041B24801F0E5
:1049000034FB0028F8D100BF1021AF4801F038FB7C
:104910004FF4005000230122D0210090AA4801F05A
:104920009CFA11E01021A84801F01FFB01280BD1CF
:1049300000BF2021A44801F018FB0028F9D0202155
:10494000A14801F01DFBDFE702219F4801F00DFBAC
:104950000028E7D080219C4801F0F8FA00BF4021F0
:10496000994801F002FB0028F9D001220421964861
:1049700001F0A3F94FF410504FF000738022D021C2
:104980000090914801F069FA08BD38B5054600BFAE
:104990004FF400418C4801F0E8FA0028F8D100BF3C
:1049A0001021894801F0ECFA4FF400500023012255
:1049B000D0210090844801F050FA11E01021824883
:1049C00001F0D3FA01280BD100BF20217E4801F06D
:1049D000CCFA0028F9D020217B4801F0D1FADFE79A
:1049E0000221794801F0C1FA0028E7D080217648F9
:1049F00001F0ACFA00BF4021734801F0B6FA00287C
:104A0000F9D04FF410504FF000738022D021009065
:104A10006D4801F022FA00241DE000BF04216A481D
:104A200001F0A3FA0028F9D0674801F091FA25F8BF
:104A3000140000BF0421644801F097FA0028F9D05F
:104A4000614801F085FA35F8141041EA002025F894
:104A50001400601CC4B2402CDFDB00BF20215A4888
:104A600001F083FA0028F9D02021574801F088FA94
:104A700038BD38B5044600BF4FF40041524801F03C
:104A800074FA0028F8D100BF10214F4801F078FADD
:104A90004FF4005000230122D02100904A4801F039
:104AA000DCF911E01021484801F05FFA01280BD130
:104AB00000BF2021444801F058FA0028F9D02021F5
:104AC000414801F05DFADFE702213F4801F04DFA6D
:104AD0000028E7D021463C4801F038FA00BF4021C9
:104AE000394801F042FA0028F9D04FF410504FF045
:104AF00000730122D0210090334801F0AEF900BFCD
:104B00000421314801F031FA0028F9D02E4801F093
:104B10001FFA054600BF20212B4801F026FA002885
:104B2000F9D02021284801F02BFA284638BD38B5A5
:104B300004460D4600BF4FF40041234801F015FA2A
:104B40000028F8D100BF10211F4801F019FA4FF4D6
:104B5000005003030222D02100901B4801F07DF990
:104B600011E01021184801F000FA01280BD100BF14
:104B70002021154801F0F9F90028F9D02021124828
:104B800001F0FEF9DFE702210F4801F0EEF90028FD
:104B9000E7D021460C4801F0D9F900BF02210A48AC
:104BA00001F0E3F90028F9D02946074801F0CEF9D1
:104BB00000BF2021044801F0D8F90028F9D02021B5
:104BC000014801F0DDF938BD0054004010B504463D
:104BD000B4F1A04F02D0FA48844209D1012108075C
:104BE00001F0FFFE00214FF0805001F0FAFE0EE0D0
:104BF000F448844202D0F448844208D10121480795
:104C000001F0EFFE00214FF0005001F0EAFE10BD70
:104C100010B502460020D068EC4B1840D1E90034B2
:104C200023438C682343CC6823430C6923434C699A
:104C300023438C6923431843D060106B20F00F008E
:104C40000B7F5B1E1843106310BD002101604160A3
:104C50008160C1600161416181610121017770471B
:104C600010B50022C26C00220B7A5B1E0C68234335
:104C70004C682343CC6843EA04230C6943EA843339
:104C80008C8A43EA04530C7E43EA8462C26410BDFA
:104C900000210160416001210172C1600161416137
:104CA0008161704710B50022B0F1A04F02D0C44B13
:104CB000984205D1C64B1A68C64B02EA030203E0CC
:104CC000C54B1A68C34B1A40D1E9003423438C68A2
:104CD0002343CC6843EA04330C7C43EA04231A439D
:104CE000B0F1A04F02D0B64B984202D1B84B1A6037
:104CF00001E0B94B1A6010BD002101604160816084
:104D0000C1600174704721B1826842F00102826083
:104D100003E0826842F0020282607047816841F0DD
:104D20000041816070470146D1F8B4007047C0F877
:104D3000B4107047826822F08042826082680A4321
:104D400082607047014600208A6812F0004F01D04F
:104D5000012000E000207047816841F0020181607D
:104D60007047014600208A6812F0020F01D001202E
:104D700000E000207047826822F04052826021B13A
:104D8000826842F08052826003E0826842F0005202
:104D90008260704710B53AB1D0F8B03001248C4031
:104DA0002343C0F8B03006E0D0F8B03001248C4086
:104DB000A343C0F8B03010BD21B1C26842F4001264
:104DC000C26003E0C26822F40012C260704721B1E1
:104DD000C26842F48042C26003E0C26822F48042AA
:104DE000C26070470A460021C16821F0E07111439A
:104DF000C160704710B5036A784C23400362036AB0
:104E000043EA01430362036A6FF30B030362036A1D
:104E10001343036210BD436A23F47F034362436A72
:104E200043EA01434362436A23F0FF034362436A58
:104E3000134343627047836A23F47F038362836A68
:104E400043EA01438362836A23F0FF038362836A38
:104E50001343836270470A460021C16821F0F8417C
:104E600041EA8261C16070470A46002150F8A01FE4
:104E70005B4B194001239340194303680B4340F8EF
:104E8000A03970470A46002150F8A41F544B19401E
:104E900001239340194303680B4340F8A43970473A
:104EA00041B14B4A126842F400024FF0A043C3F8EC
:104EB000082307E0464A126822F400024FF0A0439C
:104EC000C3F808237047B0F1A04F02D03C4A90428B
:104ED00012D141B13E4A126842F480024FF0A04321
:104EE000C3F8082316E03A4A126822F480024FF011
:104EF000A043C3F808230DE031B1374A126842F4E9
:104F00008002354B1A6005E0334A126822F48002B1
:104F1000314B1A60704741B12D4A126842F08072DD
:104F20004FF0A043C3F8082307E0294A126822F093
:104F300080724FF0A043C3F808237047F0B50C46C9
:104F40001D4600BF00BF052A0FDA016B02EB4206C7
:104F500077001F2606FA07F3994302EB4206760014
:104F600004FA06F3194301634FE00A2A11DA416B90
:104F7000561F06EB460677001F2606FA07F39943ED
:104F8000561F06EB4606760004FA06F31943416302
:104F90003BE00F2A26DA816BA2F10A0606EB4606F1
:104FA00077001F2606FA07F39943A2F10A0606EBDB
:104FB0004606760004FA06F31943816325E00000F3
:104FC00000010050000400500005005007C0FFFD24
:104FD00008030050E010FCFF08070050FFFF00F03E
:104FE0000100F8FFC16BA2F10F0606EB4606770041
:104FF0001F2606FA07F39943A2F10F0606EB4606B1
:10500000760004FA06F31943C163092C14DD8169A3
:10501000A4F10A0606EB4607072606FA07F3866997
:105020009E4386618669A4F10A0707EB470705FAE4
:1050300007F73E43866110E04169661E06EB4607AE
:10504000382606FA07F346699E434661466904EB33
:10505000440705FA07F73E434661F0BD026B22F0B4
:105060000F020263026B4B1E1A430263704710B5B6
:10507000C36823F47C63C360C36842EA010423432A
:10508000C36010BD816841F0040181607047014632
:1050900000208A6812F0040F01D0012000E00020F7
:1050A0007047816841F010018160704710B50A4671
:1050B00000210023C16821F46021531E41EA4341CD
:1050C000C16010BD21B1C26842F48032C26003E009
:1050D000C26822F48032C26070470146086C80B218
:1050E000704701460020B1F1A04F02D09F4A914283
:1050F00002D19F4A106801E09E4A10687047036E13
:1051000023F0F8430366036E43EA81630366036E8C
:105110006FF30B030366036E134303667047436E1E
:1051200023F0F8434366436E43EA81634366436E6C
:105130006FF30B034366436E134343667047836EFE
:1051400023F0F8438366836E43EA81638366836E4C
:105150006FF30B038366836E134383667047C36EDE
:1051600023F0F843C366C36E43EA8163C366C36E2C
:105170006FF30B03C366C36E1343C366704721B15D
:10518000026E42F00042026603E0026E22F000422C
:105190000266704721B1426E42F00042426603E06F
:1051A000426E22F000424266704721B1826E42F0A8
:1051B0000042826603E0826E22F0004282667047FF
:1051C00021B1C26E42F00042C26603E0C26E22F01C
:1051D0000042C266704721B1C26842F00102C2605B
:1051E00003E0C26822F00102C2607047C26822F088
:1051F0000202C260C2680A43C260704730B5002331
:10520000092913DDA1F10A0404EB4405072404FA7B
:1052100005F384699C4384618469A1F10A0505EB67
:10522000450502FA05F52C4384610FE04C1E04EBA2
:105230004405382404FA05F344699C4344614469F5
:1052400001EB410502FA05F52C43446130BD81684C
:1052500041F0080181607047816841F02001816060
:105260007047014600208A6812F0080F01D0012023
:1052700000E00020704721B1C26842F00072C260B5
:1052800003E0C26822F00072C260704721B1C268B8
:1052900042F48012C26003E0C26822F48012C2604D
:1052A000704708B50246002000900092481E8023F7
:1052B00003EB8000009B184400900098006880B2C7
:1052C00008BD1AB143680B43436002E043688B4357
:1052D000436070470246002013680B4201D0012052
:1052E00000E0002070470160704710B502460023BF
:1052F0000020B2F1A04F02D01C4CA24202D11E4CA1
:10530000236802E01B4C0C3C23680B4201D00120B7
:1053100000E0002010BDB0F1A04F02D0134A90422F
:1053200008D1154A126842EA01024FF0A043C3F8BF
:10533000002306E00F4A0C3A12680A430D4B0C3B5F
:105340001A60704730B5024600200023002415681B
:105350000D40ABB255680D40ACB213B10CB1012099
:1053600000E0002030BD01607047000000010050E7
:105370000C0300500C0700500003005001460020B1
:10538000F94A106820F0030008431060704730B1FC
:10539000F549096841F00801F34A116005E0F24956
:1053A000096821F00801F04A1160704730B1EE49F8
:1053B000096841F01001EC4A116005E0EA4909680A
:1053C00021F01001E84A11607047E748006910F0C9
:1053D000800F04D0E548E4494860E54848607047DC
:1053E000E148006940F08000DF490861704704200F
:1053F000DD49C96811F0010F01D001200EE0DA4942
:10540000C96811F0100F01D0022007E0D649C96821
:1054100011F0040F01D0032000E00420704700B514
:1054200002460423FFF7E3FF034603E0FFF7DFFF35
:105430000346521E012B01D1002AF7D102B90523E0
:10544000184600BD30B5044604254FF43020FFF760
:10545000E6FF0546042D16D1C348006940F002005E
:10546000C149086108464461006940F04000086194
:105470004FF43020FFF7D3FF0546BB48006920F00A
:105480000200B9490861284630BD10B504244FF424
:105490003020FFF7C4FF0446042C15D1B248006940
:1054A00040F00400B04908610846006940F040003F
:1054B00008614FF43020FFF7B2FF0446AA480069A4
:1054C00020F00400A8490861204610BD78B50646C2
:1054D0000C460425002000904FF43020FFF79FFF7A
:1054E0000546042D24D1A048006940F001009E49E2
:1054F000086134804FF43020FFF791FF0546042DFA
:1055000010D1B01C0090200C009908804FF430207E
:10551000FFF785FF05469448006920F00100924995
:10552000086105E09048006920F001008E4908619B
:10553000284678BD70B504460D4604264FF4302049
:10554000FFF76DFF0646042E11D18748006940F031
:1055500001008549086125804FF43020FFF75FFF87
:1055600006468148006920F001007F490861304605
:1055700070BD7D48006910F4007F04D17B487A49F2
:1055800088607B48886070477748006920F4007025
:105590007549086170477448006940F400507249C9
:1055A0000861704700207049C96911F0060F01D0E9
:1055B000012000E00020704730B5AA250424FFF741
:1055C000F1FF00B100254FF43020FFF728FF04461B
:1055D000042C34D16448006940F02000624908611D
:1055E0000846006940F0400008614FF43020FFF7A2
:1055F00016FF0446042C1AD15B48006920F02000F5
:10560000594908610846006940F01000086159488E
:1056100005804FF43020FFF702FF0446052C0ED022
:105620005148006920F010004F49086107E0052C3F
:1056300005D04D48006920F010004B490861204614
:1056400030BD2DE9F04304464FF6FF763746B046AD
:10565000B1460425E443E6B2C4F30727C4F3074880
:105660004FEA14694FF43020FFF7D9FE0546042DA8
:105670003FD13D48006940F010003B490861FF2ED2
:1056800007D03C48083006804FF43020FFF7C7FEB3
:105690000546042D09D1FF2F07D036480A30078070
:1056A0004FF43020FFF7BBFE0546042D0BD1B8F1B7
:1056B000FF0F08D02F480C30A0F800804FF43020A6
:1056C000FFF7ADFE0546042D0BD1B9F1FF0F08D051
:1056D00028480E30A0F800904FF43020FFF79FFECE
:1056E0000546052D05D02048006920F010001E4910
:1056F00008612846BDE8F08330B5054604244FF420
:105700003020FFF78CFE0446042C3DD1164800697A
:1057100040F02000144908610846006940F040004C
:1057200008614FF43020FFF77AFE0446042C23D1A1
:105730000D48006920F020000B4908610846006907
:1057400040F0100008610B4805804FF43020FFF74F
:1057500066FE0446052C17D00348006920F01000AF
:105760000149086110E00000002002402301674564
:10577000AB89EFCD00F8FF1F052C05D089480069E3
:1057800020F0200087490861204630BDF0B507466B
:105790000D46164604248448824988608348886000
:1057A0004FF43020FFF73BFE0446042C19D17D480E
:1057B000006940F010007B49086147EA050046F0A7
:1057C000F80108437A4908804FF43020FFF727FE9C
:1057D0000446052C05D07348006920F0100071497B
:1057E00008612046F0BD30B5054604246E486D4979
:1057F00088606E4888604FF43020FFF710FE044642
:10580000042C16D16748006940F010006549086112
:1058100045F0EF00664908804FF43020FFF7FFFDA8
:105820000446052C05D05F48006920F010005D4952
:105830000861204630BD30B5054604245A48594910
:1058400088605A4888604FF43020FFF7E8FD04462E
:10585000042C16D15348006940F0100051490861EA
:1058600045F0DF00524908804FF43020FFF7D7FDA4
:105870000446052C05D04B48006920F0100049492A
:105880000861204630BD30B5054604244FF4302071
:10589000FFF7C5FD0446042C16D14248006940F0CC
:1058A00010004049086145F0BF00414908804FF4AD
:1058B0003020FFF7B4FD0446052C05D039480069B7
:1058C00020F0100037490861204630BD30B505464C
:1058D0000424354833498860344888604FF43020C8
:1058E000FFF79DFD0446042C16D12E48006940F0B8
:1058F00010002C49086145F088002D4908804FF4BC
:105900003020FFF78CFD0446052C05D025480069A2
:1059100020F0100023490861204630BD70B50546CF
:105920000E4604244FF43020FFF779FD0446042C82
:1059300013D11C48006940F010001A4908612E80FC
:105940004FF43020FFF76BFD0446052C05D01548B9
:10595000006920F0100013490861204670BD11480D
:10596000C069C0F3072070470E48006A704729B12C
:105970000C4A126902430B4B1A6104E0094A12698E
:105980008243084B1A61704701460020054AD268DD
:105990000A4201D0012000E0002070470149C860A0
:1059A000704700000020024023016745AB89EFCD1E
:1059B00002F8FF1F10B50446B4F1904F09D1012140
:1059C000480401F00EF800214FF4003001F009F80E
:1059D00056E07E48844208D10121000201F001F81E
:1059E0000021200200F0FDFF4AE07948844208D1FE
:1059F0000121000200F0F5FF0021200200F0F1FF7C
:105A00003EE07448844209D10121080500F0E9FF15
:105A100000214FF4801000F0E4FF31E06E48844232
:105A200008D10121400200F0DCFF0021600200F0FB
:105A3000D8FF25E06948844209D10121880500F09A
:105A4000D0FF00214FF4800000F0CBFF18E0644845
:105A5000844209D10121C80500F0C3FF00214FF4A1
:105A6000000000F0BEFF0BE05E48844208D1012137
:105A7000080400F0B6FF00214FF4803000F0B1FFC1
:105A800010BDF0B50A46002100240025002300BF08
:105A90003FE0012606FA01F4166806EA0405A5426D
:105AA00036D11679012E02D01679022E18D18668C9
:105AB0004FEA410C032707FA0CF7BE43866056797C
:105AC0004F00BE4087683E438660868801278F402E
:105AD000BE438680878896798E40B6B237438780EA
:105AE00006684FEA410C032707FA0CF7BE4306602D
:105AF00016794F00BE4007683E430660C3684F00FA
:105B00000326BE40B343D6794F00BE403343C36043
:105B1000491C1029BDD3F0BD4FF6FF710160002173
:105B200001710221417100218171C17170474FF4EF
:105B300080320A43C261C161C261C269C2697047F1
:105B400002460020138A0B4201D0012000E0002011
:105B500070470146088A704702460020938A0B422C
:105B600001D0012000E0002070470146888A70477C
:105B700081617047018570470AB1816100E001854C
:105B8000704781827047F0B5002300244D07ED0E69
:105B900002FA05F3CE1000F1200555F826504E0705
:105BA000F70E0F26BE40B543CF1000F1200646F891
:105BB0002750CE1000F1200555F8265045EA030481
:105BC000CE1000F1200545F82640F0BD0004004845
:105BD00000080048000C004800100048001400486D
:105BE00000180048001C004810B50446F5488442DF
:105BF00009D10121480500F00EFF00214FF40010EB
:105C000000F009FF08E00121880500F004FF0021F1
:105C10004FF4800000F0FFFE10BD10B50A460021D1
:105C2000036823F0010303600168E74B1940D2E9E0
:105C3000013443EA042319430160136823F07063BD
:105C40000361036843F00103036000218160C160C8
:105C50001469936943EA04018160836843F4004353
:105C60008360D16803680B4303604168D74B1940D8
:105C700053691943416010BD00210160416081609A
:105C8000C16001614FF400414161002181617047B1
:105C900021B1026842F00102026003E0026822F0D2
:105CA000010202607047016821F001010160016892
:105CB000016841F00101016070471AB103680B43AC
:105CC000036002E003688B430360704721B1026800
:105CD00022F40032026003E0026842F40032026003
:105CE000704721B1026842F48022026003E002683A
:105CF00022F480220260704721B1C26842F400425F
:105D0000C26003E0C26822F40042C260704730B54E
:105D10000B460021C16840F2FE74A14303F0FE046B
:105D20004FF4E06505EA02252C432143C16030BDF4
:105D300021B1026842F40022026003E0026822F40A
:105D400000220260704721B1026842F48032026092
:105D500003E0026822F48032026070470A460021A4
:105D600041686FF30901C2F30903194341607047A9
:105D700021B1426842F40062426003E0426822F4CA
:105D800000624260704721B1426842F00072426096
:105D900003E0426822F000724260704721B142681D
:105DA00042F08072426003E0426822F080724260FA
:105DB00070470A460021416821F47F014FF47F03B8
:105DC00003EA024319434160704721B9426822F453
:105DD0008062426003E0426842F480624260704741
:105DE00021B1426842F40052426003E0426822F46A
:105DF00000524260704721B1426842F480424260E2
:105E000003E0426822F480424260704721B1426858
:105E100042F48052426003E0426822F480524260C1
:105E2000704721B1426822F40042426003E04268B8
:105E300042F40042426070470146886900F47E00E7
:105E4000000C70470146002200208B6903F4803269
:105E500002B901E04FF480607047F0B50C46059D33
:105E6000002141685A4E3140C4F309064FF47F07C0
:105E700007EA02473E431E432E4331434160F0BDD3
:105E800021B1026842F48002026003E0026822F459
:105E900080020260704721B1426942F400424261CF
:105EA00003E0426922F400424261704721B1426935
:105EB00042F00042426103E0426922F00042426146
:105EC000704721B1426942F48052426103E0426965
:105ED00022F48052426170470A46002141696FF303
:105EE0000B01C2F30B031943416170470A460021BD
:105EF0004169384B1940DB4303EA024319434161CE
:105F0000704721B1026842F40002026003E00268B7
:105F100022F400020260704721B1026842F0806200
:105F2000026003E0026822F080620260704701466E
:105F3000086AC0B2704708B502460020009000927F
:105F40000098084400900098006808BD816270477E
:105F50000146486AC0B270471AB103680B43036038
:105F600002E003688B430360704710B502460023CC
:105F7000002093690B400BB1012000E0002010BD10
:105F8000C161704730B5024600230020002411F49F
:105F90007C5F03D0156805F0800409E011F0C00FA4
:105FA00003D0156805F0400402E0156805EA010415
:105FB00093690B4013B10CB1012000E0002030BD0B
:105FC000C161704700540040FFE0CF00FF7FFF0732
:105FD000009800FCFFFF00F031490143314A116095
:105FE000704770B5002100230F22C4780CB32D4CEC
:105FF000246804F4E064C4F5E064210AC1F10403F8
:10600000CA40447804FA03F184781440214309011A
:10601000254C0678A155047804F01F050124AC40F6
:1060200005786D114FF0E02606EB8505C5F80041B7
:1060300009E0047804F01F050124AC401B4D0678EC
:10604000761145F8264070BD194A0A400243154BA7
:106050001B1F1A60704739B1124A121D12680243A1
:10606000104B1B1D1A6006E00E4A121D1268824377
:106070000C4B1B1D1A607047042808D14FF0E0211B
:10608000096941F004014FF0E022116107E04FF08F
:10609000E021096921F004014FF0E022116170470D
:1060A0000000FA050CED00E000E400E080E100E013
:1060B00080FFFF1FFE48006840F00100FC490860B7
:1060C00008464068FB490840F949486008460068AE
:1060D000F9490840F64908600846006820F4802025
:1060E00008600846406820F4FE0048600846C06A20
:1060F0006FF30D00C8620846006BF0490840EC4998
:1061000008630020886070470021E94A91701146B9
:106110008870704710B502460021002300205111FD
:1061200011B9E34C23680BE0012902D1E04C236A4A
:1061300006E0042902D1DE4C636801E0DC4C636AAE
:1061400002F01F0101248C401C4201D0012000E01C
:10615000002010BD38B5002000900024002500BFAD
:106160001120FFF7D7FF05460098401C00900098CB
:10617000B0F5A04F01D0002DF2D01120FFF7CAFFDB
:1061800008B1012400E00024204638BD014600206B
:10619000C74A106820F0F80040EAC100106070475C
:1061A000C74908607047C249096A21F00101C04A25
:1061B00011621146096A21F0040111621146096A4F
:1061C000014311627047BA49096A21F01801B84ABF
:1061D00011621146096A014311627047B9490860AA
:1061E0007047B34A526822F47412B14B5A601A468F
:1061F000526840EA01031A43AD4B5A607047B049F8
:106200000866704701460020A94AD06A20F00F00B6
:106210000843D0627047AA49C8647047014600200D
:10622000A34A506820F0074040EA01605060704780
:10623000014600209E4A506820F003000843506049
:1062400070479B48406800F00C00704701460020F2
:10625000974A506820F0F0000843506070470146AC
:106260000020934A506820F4E06008435060704773
:10627000014600208E4A506820F4605040EAC10078
:10628000506070472DE9F043002200260027944615
:106290000025002100230024DFF81482D8F80480B0
:1062A00008F00C0222B1042A07D0082A30D109E0F4
:1062B000DFF81482C0F800802FE0DFF80C82C0F80D
:1062C00000802AE0DFF8E881D8F8048008F470162E
:1062D000DFF8DC81D8F8048008F480374FF002083A
:1062E00008EB964627B9DFF8E48106FB08F10DE0DC
:1062F000DFF8BC81D8F82C8008F00F0808F1010CF9
:10630000DFF8C481B8FBFCF808FB06F1016004E08B
:10631000DFF8B481C0F8008000BF00BFDFF89081D3
:10632000D8F8048008F0F0021209DFF8A48118F808
:106330000240D0F8008028FA04F8C0F80480DFF8A2
:106340007081D8F8048008F4E062120ADFF88081D6
:1063500018F80250D0F8048028FA05F8C0F8088030
:10636000DFF84C81D8F8048008F46052D20ADFF8D4
:10637000608118F80230D0F8048028FA03F8C0F8D9
:106380000C80DFF82C81D8F82C8008F4F872120900
:1063900002F00F08DFF83C9139F8185012F0100F96
:1063A00005D025B1B1FBF5F8C0F8108003E0D0F8B6
:1063B0000080C0F81080DFF8F880D8F82C8008F44E
:1063C0007852520A02F00F08DFF8089139F8185095
:1063D00012F0100F05D025B1B1FBF5F8C0F814800C
:1063E00003E0D0F80080C0F81480DFF8C480D8F84B
:1063F000308008F01008B8F1100F04D0DFF8C88022
:10640000C0F8188003E0D0F80080C0F81880DFF8EA
:10641000A080D8F8308008F02008B8F1200F04D010
:10642000DFF8A480C0F81C8003E0D0F80080C0F83A
:106430001C80DFF87C80D8F8308008F04008B8F184
:10644000400F04D0DFF88080C0F8208003E0D0F84F
:106450000080C0F82080DFF85880D8F8308008F439
:106460008078B8F5807F0AD1D0F80080884506D1C1
:10647000A34204D14FEA4108C0F8248003E0D0F8D9
:106480000C80C0F82480DFF82880D8F8308008F429
:106490008058B8F5805F1FD1D0F8008088451BD1A7
:1064A000A34219D14FEA4108C0F8288018E0000043
:1064B0000010024000C0FFF8FFFFF6FECCEC000F1A
:1064C000000042428004424200127A0000093D006E
:1064D0006400002074000020D0F80C80C0F82880F0
:1064E000DFF89085D8F8308008F40078B8F5007FA0
:1064F0000AD1D0F80080884506D1A34204D14FEAE2
:106500004108C0F82C8003E0D0F80C80C0F82C8043
:10651000DFF86085D8F8308008F48068B8F5806FBF
:106520000AD1D0F80080884506D1A34204D14FEAB1
:106530004108C0F84C8003E0D0F80C80C0F84C80D3
:10654000DFF83085D8F8308008F40068B8F5006FBF
:106550000AD1D0F80080884506D1A34204D14FEA81
:106560004108C0F8508003E0D0F80C80C0F850809B
:10657000DFF80085D8F8308008F40058B8F5005FDF
:106580000AD1D0F80080884506D1A34204D14FEA51
:106590004108C0F8548003E0D0F80C80C0F8508067
:1065A000DFF8D084D8F8308008F40048B8F5004F00
:1065B0000AD1D0F80080884506D1A34204D14FEA21
:1065C0004108C0F8588003E0D0F80C80C0F858802B
:1065D000DFF8A084D8F8308018F0030F04D1D0F889
:1065E0000C80C0F8388028E0DFF88884D8F8308044
:1065F00008F00308B8F1010F04D1D0F80080C0F80A
:1066000038801AE0DFF86C84D8F8308008F003088E
:10661000B8F1020F04D14FF40048C0F838800CE004
:10662000DFF85084D8F8308008F00308B8F1030F81
:1066300003D1DFF84484C0F83880DFF83884D8F814
:10664000308018F4403F04D1D0F80880C0F83C8076
:1066500028E0DFF82084D8F8308008F44038B8F516
:10666000803F04D1D0F80080C0F83C801AE0DFF809
:106670000484D8F8308008F44038B8F5003F04D1DD
:106680004FF40048C0F83C800CE0DFF8E883D8F80D
:10669000308008F44038B8F5403F03D1DFF8D883A4
:1066A000C0F83C80DFF8CC83D8F8308018F4402F55
:1066B00004D1D0F80880C0F8408028E0DFF8B48327
:1066C000D8F8308008F44028B8F5802F04D1D0F8ED
:1066D0000080C0F840801AE0DFF89883D8F8308056
:1066E00008F44028B8F5002F04D14FF40048C0F852
:1066F00040800CE0DFF87C83D8F8308008F4402834
:10670000B8F5402F03D1DFF87083C0F84080DFF880
:106710006483D8F8308018F4401F04D1D0F8088082
:10672000C0F8448028E0DFF84C83D8F8308008F4C3
:106730004018B8F5801F04D1D0F80080C0F844801C
:106740001AE0DFF83083D8F8308008F44018B8F544
:10675000001F04D14FF40048C0F844800CE0DFF87B
:106760001483D8F8308008F44018B8F5401F03D1DE
:10677000DFF80483C0F84480DFF8F882D8F830806E
:1067800018F4400F04D1D0F80880C0F8488028E001
:10679000DFF8E082D8F8308008F44008B8F5800FC0
:1067A00004D1D0F80080C0F848801AE0DFF8C48235
:1067B000D8F8308008F44008B8F5000F04D14FF441
:1067C0000048C0F848800CE0DFF8A882D8F8308094
:1067D00008F44008B8F5400F03D1DFF89C82C0F8F8
:1067E0004880BDE8F0830021010F31B1A14AD26A8F
:1067F00022F478529F4BDA6205E09E4AD26A22F474
:10680000F8729C4BDA629B4AD26A0243994BDA6275
:1068100070470021010F21B1012909D0022915D1AA
:106820000DE0944A126B22F01002924B1A630EE0B4
:10683000904A126B22F020028E4B1A6307E08D4AB9
:10684000126B22F040028B4B1A6300E000BF00BFC6
:10685000884A126B0243874B1A6370470021010F6D
:1068600008293DD2DFE801F0040B121920272E354C
:10687000804A126B22F480727E4B1A6331E07D4AAB
:10688000126B22F400727B4B1A632AE0794A126B76
:1068900022F48062774B1A6323E0764A126B22F46B
:1068A0000062744B1A631CE0724A126B22F40052AD
:1068B000704B1A6315E06F4A126B22F400426D4B65
:1068C0001A6300BF6B4A126B22F08072694B1A6325
:1068D00000BF684A126B22F00072664B1A6300E038
:1068E00000BF00BF634A126B0243624B1A637047DA
:1068F0006049096B21F480515E4A11631146096BAE
:106900000143116370470021010F062927D2DFE8F8
:1069100001F026030A11181F564A126B22F00302D7
:10692000544B1A631CE0534A126B22F44032514B11
:106930001A6315E04F4A126B22F440224D4B1A6342
:106940000EE04C4A126B22F440124A4B1A6307E0E5
:10695000484A126B22F44002464B1A6300E000BF23
:1069600000BF444A126B0243424B1A6370474349CB
:10697000086070473F49096A01433E4A1162704707
:106980003F49086070473F49086070473D49091D0D
:106990000860704729B1374A52690243354B5A6142
:1069A00004E0344A52698243324B5A61704729B13C
:1069B000304A926902432F4B9A6104E02D4A926952
:1069C00082432C4B9A61704729B12A4AD26902430B
:1069D000284BDA6104E0274AD2698243254BDA6109
:1069E000704729B1234A926A0243224B9A6204E01B
:1069F000204A926A82431F4B9A62704729B11D4A0E
:106A0000D26802431B4BDA6004E01A4AD268824320
:106A1000184BDA60704729B1164A12690243154BC8
:106A20001A6104E0134A12698243124B1A617047DB
:106A300029B1104A527A02430E4B5A7204E00D4AB1
:106A4000527A82430B4B5A7270470A48406A40F0B0
:106A5000807008494862704701460020054A9268E4
:106A60000A4201D0012000E00020704701498872ED
:106A7000704700000010024000127A00D800424225
:106A8000DC0042423C04424210B50446FE488442C7
:106A900008D10121C014FFF7B1FF0021E014FFF776
:106AA000ADFF7AE0B4F1804F08D101210846FFF72D
:106AB000B2FF00210120FFF7AEFF6EE0F3488442F1
:106AC00008D101210220FFF7A6FF00210220FFF7D5
:106AD000A2FF62E0EE48844208D101210420FFF7C2
:106AE0009AFF00210420FFF796FF56E0E948844210
:106AF00008D101211020FFF78EFF00211020FFF7A1
:106B00008AFF4AE0E448844208D101212020FFF7AF
:106B100082FF00212020FFF77EFF3EE0DF48844215
:106B200008D101214014FFF769FF00216014FFF72D
:106B300065FF32E0DA48844209D101210804FFF7F9
:106B40005DFF00214FF48030FFF758FF25E0D54866
:106B5000844209D101214804FFF750FF00214FF47E
:106B60000030FFF74BFF18E0CF48844209D10121E4
:106B70008804FFF743FF00214FF48020FFF73EFF1A
:106B80000BE0CA48844208D101210805FFF736FF0F
:106B900000214FF48010FFF731FF10BD0022028862
:106BA000B94B98420ED0BD4B98420BD0B0F1804FFC
:106BB00008D0B64B984205D0B54B984202D0BB4B9B
:106BC000984204D14FF68F731A404B881A43B14B49
:106BD000984207D0B04B984204D04FF6FF431A407A
:106BE0000B891A4302804B68C3620B880385A64B4E
:106BF00098420ED0A94B98420BD0A94B984208D08E
:106C0000A84B984205D0A84B984202D0A74B984277
:106C100001D14B8903860123436170474FF0FF3157
:106C200041600021018001814180418170470185DF
:106C3000426170470A46002101884FF68F73194060
:106C400011430180704741627047C162704701463D
:106C5000486A70470146088D704721B1028842F0AA
:106C60000202028004E002884FF6FD731A4002809F
:106C7000704721B1028842F00402028004E00288D9
:106C80004FF6FB731A400280704721B1028842F42C
:106C90000062028004E002884FF2FF731A40028013
:106CA000704721B1028842F08002028004E002882D
:106CB0004FF67F731A400280704702884FF6F773D1
:106CC0001A40028002880A430280704702884FF609
:106CD000FF431A40028002880A430280704721B1B4
:106CE000028842F00102028004E002884FF6FE733F
:106CF0001A400280704730B5002400220023056A44
:106D000025F001050562026A43688469684D2C40DC
:106D100024F003040D682C4322F002028D892A43DB
:106D20008D882A43584DA8420BD05C4DA84208D00C
:106D30005B4DA84205D05B4DA84202D05A4DA842F7
:106D40000FD122F00802CD892A4322F00402CD8817
:106D50002A4323F4807323F400730D8A2B434D8A56
:106D60002B43436084618D684563026230BD30B55A
:106D7000002400220023056A25F010050562026A3E
:106D8000436884694B4D2C4024F440740D6844EAF8
:106D9000052422F020028D8942EA05128D8842EAFC
:106DA0000512394DA84202D03C4DA84213D122F021
:106DB0008002CD8942EA051222F04002CD8842EAE3
:106DC000051223F4806323F400630D8A43EA8503EC
:106DD0004D8A43EA8503436084618D68856302625E
:106DE00030BD30B5002400220023056A25F48075EB
:106DF0000562026A4368C46924F0700424F0030445
:106E00000D682C4322F400728D8942EA05228D8898
:106E100042EA05221C4DA84202D0204DA84213D1BF
:106E200022F40062CD8942EA052222F48062CD88F4
:106E300042EA052223F4805323F400530D8A43EAE7
:106E400005134D8A43EA05134360C4618D68C56329
:106E5000026230BD30B5002200230024056A25F40B
:106E600080550562036A4468C26922F4E04222F454
:106E700040720D6842EA052223F400538D8943EAEB
:106E800005338D8818E00000002C0140000400400C
:106E90000008004000100040001400400034014091
:106EA00000400140004401400048014000500140C2
:106EB0008FFFFEFFFF8FFFFE43EA0533F84DA84228
:106EC00002D0F84DA84204D124F480440D8A44EA4B
:106ED00085144460C2618D680564036230BD30B5BD
:106EE000002300220024056A25F480350562026A29
:106EF0004468436D23F070030D682B4322F4003285
:106F00008D8942EA05428D8842EA0542E44DA84255
:106F100002D0E44DA84204D124F480340D8A44EA1E
:106F20000544446043658D688565026230BD70B577
:106F3000002300220024056A25F480150562026AF8
:106F40004468436D23F4E0430D6843EA052322F4CB
:106F500000128D8942EA05528D8842EA0552D04DD1
:106F6000A84202D0CF4DA84207D124F400340D8AA4
:106F70004FF6FF7606EA85452C43446043658D68ED
:106F8000C565026270BD21B1826D42F0005282651A
:106F900003E0826D22F000528265704721B1826D5C
:106FA00042F08042826503E0826D22F08042826579
:106FB000704721B1826D42F00042826503E0826D2C
:106FC00022F0004282657047002101608180C1800B
:106FD00081608181C18101824182704770B5034621
:106FE000002000241846183001258D40ACB21D6ADF
:106FF000E643B6B235401D6209B1082909D100EB5C
:1070000061000568A84E35400560056815430560B8
:107010000AE00D1F00EB55000568A44E35400560E1
:10702000056845EA0225056070BD416370478163CC
:107030007047C16370470164704781657047C165DF
:1070400070470A4600218169974B194011438161BD
:1070500070470A4600218169944B194041EA022198
:10706000816170470A460021C16921F07001114316
:10707000C16170470A460021C16921F4E04141EA3B
:107080000221C16170470A460021416D21F0700163
:107090001143416570470A460021416D21F4E041EA
:1070A00041EA0221416570470A460021816921F0C9
:1070B00008011143816170470A460021816921F46A
:1070C000006141EA0221816170470A460021C169DD
:1070D00021F008011143C16170470A460021C169CE
:1070E00021F4006141EA0221C16170470A46002192
:1070F000416D21F008011143416570470A460021A6
:10710000416D21F4006141EA0221416570470A4660
:107110000021816921F004011143816170470A4611
:107120000021816921F4806141EA02218161704777
:107130000A460021C16921F004011143C161704771
:107140000A460021C16921F4806141EA0221C1613E
:1071500070470A460021816921F080011143816155
:1071600070470A460021816921F4004141EA022169
:10717000816170470A460021C16921F080011143F5
:10718000C16170470A460021C16921F4004141EA0A
:107190000221C16170470A460021416D21F0800142
:1071A0001143416570470A460021416D21F40041B9
:1071B00041EA02214165704782684FF6F7731A4031
:1071C000826082680A43826070470A460021016A31
:1071D00021F002011143016270470A460021016A51
:1071E00021F008011143016270470A460021016A3B
:1071F00021F0200141EA0211016270470A46002194
:10720000016A21F0800141EA0211016270470A46D9
:107210000021016A21F4007141EA022101627047F4
:107220000A460021016A21F4006141EA022101625B
:1072300070470A460021016A21F4005141EA0231F7
:10724000016270470A460021016A21F4003141EAD7
:107250000241016270470A460021016A21F40011CF
:1072600041EA02510162704730B50023012404FA5B
:1072700001F3046A9C430462046A02FA01F52C4398
:10728000046230BD30B50023042404FA01F3046A1B
:107290009C430462046A02FA01F52C43046230BD87
:1072A000002C0140003401408FFFFEFFFF8FFFFEE6
:1072B000C2694FF2FF331A40C261C2694FF6FF73D1
:1072C00003EA01231A43C2617047F0B50C46154624
:1072D000002100220026076A4EF6FF7C07EA0C0711
:1072E0000762C769B9B2076ABAB24FF6FF7707EA11
:1072F000043640F6FF4739404FF6FF7707EA052787
:1073000039434FF6FF7707EA0337394345F6FF77EE
:107310003A4046F480573A43C1610262F0BDC26907
:107320004FF6F3731A40C261C2690A43C2617047E3
:10733000F0B50C461546002100220026076A4FF6DC
:10734000FF6C07EA0C070762C769B9B2076ABAB2ED
:107350004FF6FF7707EA04264FF60C7739404FF6D1
:10736000FF7707EA03172F4339434FF2FF573A409D
:1073700046F480773A43C1610262F0BD826922F42B
:1073800040628261826942EA012282617047F0B5FF
:107390000C461546002100220026076A4FF6EF7CB6
:1073A00007EA0C0707628169026A4FF6FF7707EA6E
:1073B000041621F4734141EA033141EA05214FF6F5
:1073C0005F773A4046F010073A4381610262F0BDB0
:1073D000826922F00C02826182690A4382617047ED
:1073E00070B50C46154600210022066A26F00106FB
:1073F00006628169026A21F0F30145EA031631430E
:1074000022F00A0244F0010632438161026270BD3B
:1074100070B505460C46208850B92389A28861883A
:107420002846FFF7DDFFE1882846FFF7D1FF25E07A
:10743000208804280AD12389A28861882846FFF77A
:10744000A6FFE1882846FFF799FF17E02088082863
:107450000AD12389A28861882846FFF769FFE1885D
:107460002846FFF75CFF09E02389A2886188284647
:10747000FFF72BFFE1882846FFF71AFF70BD0021B8
:1074800001804180012181800021C18001817047FC
:107490002DE9F04105460C4600260127608808B911
:1074A000022600E00026A088012801D1022700E082
:1074B00001272088A0B92389A28861882846FFF780
:1074C0008FFFE1882846FFF783FF23893A4631463C
:1074D0002846FFF75CFFE1882846FFF74FFF13E0DF
:1074E0002389A28861882846FFF751FFE188284652
:1074F000FFF744FF23893A4631462846FFF770FFDD
:10750000E1882846FFF764FFBDE8F0810146486B3B
:1075100070470146886B70470146C86B704701464B
:10752000086C70470A884B881A438B881A43CB88AB
:107530001A430B891A434B891A438B891A434264B5
:10754000704710B5436C23F472234364436C41EAE3
:1075500002442343436410BD10B5436C23F03C73D5
:107560004364436C41EA02542343436410BD21B198
:10757000426C42F48052426403E0426C22F4805236
:107580004264704721B1426C42F08072426403E071
:10759000426C22F080724264704700210180418079
:1075A0008180C180018141818181704721B1426C1C
:1075B00042F40042426403E0426CC2F30E024264B1
:1075C000704721B1426842F00402426004E0426820
:1075D0004FF6FB731A404260704721B1426842F097
:1075E0000102426004E042684FF6FE731A404260B6
:1075F000704710B51AB1C3680B43C36004E0C36899
:10760000CC43A4B22340C36010BD41617047024621
:10761000002013690B4201D0012000E000207047D8
:10762000CA4392B20261704730B50246002000237F
:107630000024156905EA0103D56805EA010413B1C0
:107640000CB1012000E0002030BDCA4392B20261BB
:10765000704741EA0203A0F84830704710B51AB1EC
:10766000C3680B43C36004E0C368CC43A4B22340A7
:10767000C36010BD21B1426842F00802426004E0DC
:1076800042684FF6F7731A404260704781684FF6C0
:10769000F8721140816070470A460021836899B2F0
:1076A0004FF68F73194011438160704730B504461F
:1076B0000D4629462046FFF7EFFFA06840F007007F
:1076C000A06030BD2DE9F04104460D4616461F4628
:1076D000602D06D13B46012231462046FFF757FE7A
:1076E00005E03B46012231462046FFF779FE294658
:1076F0002046FFF7D1FFA06840F00700A060BDE87A
:10770000F08130B50C4600218568A9B2C9B24FF6A8
:10771000FF7505EA0325154325432943816030BDE4
:107720002DE9F04105460E4617469846002443468B
:107730003A4631462846FFF7E4FFA86884B24FF680
:10774000F870044044F007044FF68F70044044F092
:107750007004AC60BDE8F081F0B504460D461646F5
:107760001F463B46324629462046FFF7CAFFA0681F
:1077700040F48040A060F0BD42684FF68F731A401D
:10778000426042680A4342607047426822F47002D5
:10779000426042680A43426070478268214B1A4047
:1077A000826082680A438260704782684FF67F7306
:1077B0001A40826082680A4382607047F0B50C46C6
:1077C00015461E460021002200238768B9B287694A
:1077D000BAB2076ABBB24FF6F877394021434FF689
:1077E000FC473A4040F201173A434FF6DD773B4001
:1077F0004FF6FF7707EA06172F433B43816082610C
:107800000362F0BD21B1426842F08002426004E0B0
:1078100042684FF67F731A4042607047A0F85010DC
:1078200070470000F8FFFEFF0CB5002001900090AB
:107830001220574908605748406856494860084632
:10784000406848600846406820F47C10486008465C
:10785000406840F4601048600846006840F080705E
:10786000086000BF4B48006810F0007FFAD049481C
:10787000406820F00300474948600846406840F0EF
:107880000200486000BF4348406800F00C00082830
:10789000F9D10CBD10B54048006840F470003E4975
:1078A00008603C48006840F001003A49086008461A
:1078B00040683A49084037494860084600683849F6
:1078C0000840344908600846006820F480200860B9
:1078D0000846406820F4FE0048600846C06A20F070
:1078E0000F00C8620846006B2E490840294908630A
:1078F00000208860FFF798FF4FF00060264980392C
:10790000086010BD30B50021002000220023214C6A
:10791000646804F00C0121B1042906D0082925D19E
:1079200007E0214C214D2C6024E01F4C1F4D2C60A2
:1079300020E0184C646804F47010164C646804F479
:107940008032022404EB904022B9194C4443174D75
:107950002C600AE00F4CE46A04F00F04631C124C24
:10796000B4FBF3F44443114D2C6003E00E4C0F4D77
:107970002C6000BF00BF074C6468C4F303140D4DB6
:10798000295D0A4C2468CC40084D2C6030BD0000B5
:10799000002002400010024088ED00E00CC07FF89B
:1079A000FFFFF6FECCFC00FF00127A0094000020DE
:1079B00000093D0098000020094880470948004719
:1079C000FEE7FEE7FEE7FEE7FEE7FEE7FEE7FEE78F
:1079D000FEE7FEE704480549054A064B70470000EC
:1079E0009578000889010008D04D0020D053002070
:1079F000D04F0020D04F00200FB41CB5074B06AA73
:107A00007B4469460090059800F07BF900206946A8
:107A100000F08AF91CBC5DF814FB0000250300008F
:107A200070B5044685690068C10601D5302600E0BE
:107A30002026C00708D070BDD4E901213046904708
:107A4000206A00F1010020626D1EF5D570BD70B591
:107A5000044685690078C00708D170BDD4E90121CA
:107A600020209047206A00F1010020626D1EF5D5AC
:107A700070BD00002DE9F04106460024106875290C
:107A8000314616A511D0AFF30080002803DAC0F10B
:107A9000000013A507E031688A0701D511A502E0AF
:107AA000490704D510A5012401E0AFF300800021AF
:107AB0000A2306F1240707E0B0FBF3F203FB1200F0
:107AC000303078541046491C0028F5D123462A4608
:107AD0003046BDE8F04100F0B2B800000000000000
:107AE0002D0000002B000000200000002DE9F047D1
:107AF0004FF0000A89460446C0F820A02046E168FD
:107B00008847002876D0252806D0D4E9012190475F
:107B1000206A401C2062F1E7E16820460025884782
:107B2000C4F81CA006460027C4F818A02A2E09D0C5
:107B3000304600F034F938B304EB8708303EC8F81B
:107B4000186019E059F8041B204604EB8702916184
:107B5000E1688847012F064618D1E069002820DA3D
:107B600025F020051DE0D8F8180000EB800006EB9A
:107B700040003038C8F818002046E16888470646BB
:107B800000F00DF90028EED1012F0AD02E2E08D1D9
:107B90002046E16888477F1C0646022F45F02005F5
:107BA000C4DBA069002803DA404245F00105A0616A
:107BB000E80701D025F01005B6B1A6F1410019285B
:107BC00002D8203645F400654A46314620462560F5
:107BD0004D46F8F713FB58B1012806D0ED1D25F0EE
:107BE000070000F1080989E704E005F1040985E7C9
:107BF00030468AE7206ABDE8F08710B5431C02E0F2
:107C000010F8011B71B18107FAD14FF0013202C89F
:107C10008C1A8C4314EAC211F9D0C01A0A0603D098
:107C2000C01E10BDC01A10BD0A0401D0801E10BDB8
:107C30000902FCD0401E10BD7047704770472DE907
:107C4000F0470D4699469246044600F12408016823
:107C5000880604D5E06921F01001216000E00120D0
:107C6000A84202DDA0EB050700E00027A16907EBB1
:107C7000050202EB0900A1EB0000A0612078C0061C
:107C800002D42046FFF7CCFE002608E0D4E901210B
:107C90001AF806009047206A401C761C20624E4568
:107CA000F4DB2078C0060AD52046FFF7B9FE06E0CF
:107CB000D4E9012130209047206A401C2062381E00
:107CC000A7F10107F4DC07E0D4E9012118F8050069
:107CD0009047206A401C2062281EA5F10105F3DCB4
:107CE0002046FFF7B4FE2078000602D50220BDE84A
:107CF000F0870120FBE7000001694A1C0261087857
:107D0000704700B58FB0CDE90131002105910549DB
:107D10007944CDE9031011466846FFF7E7FE0FB03E
:107D200000BD0000E5FFFFFF0A6802F8010B0A60D2
:107D30007047754600F028F8AE4605006946534680
:107D400020F00700854618B020B5FFF743FEBDE8D8
:107D500020404FF000064FF000074FF000084FF0B2
:107D6000000B21F00701AC46ACE8C009ACE8C00943
:107D7000ACE8C009ACE8C0098D4670470446AFF3D3
:107D800000802046F8F751FA00487047704D0020F7
:107D900001491820ABBEFEE72600020070473038CC
:107DA0000A2801D201207047002070474FF0407030
:107DB000E1EE100A70470000000000000000000023
:107DC00000000000000000000000F80000000000BB
:107DD000000019000000000000780078000000009A
:107DE0000000000000000040C07840E07840021A27
:107DF00007021E03020000E09010FC101020000893
:107E000011117F11130E304848308080400000026D
:107E100001010C12120C0000F0C808080000000F4D
:107E2000181011160817000000007800000000006C
:107E3000000000000000000000E01C040000000042
:107E40000007182000000000041CE00000000000F3
:107E50002038070000000090A060F860A0900000AB
:107E600000000100000000000000E0000000000130
:107E700001010F01010100000000FE0000000000F0
:107E80000000FF00000000000000000000000000F3
:107E900002020202000000000000000000000000DA
:107EA000001818000000000000008070080000406A
:107EB00038060100000000E01008880810E0000704
:107EC00008101010080700001008F800000000005B
:107ED00010101F10100000100808080898700010FB
:107EE00018141213111000100888888848700008B0
:107EF00010101010190F000080603008F800000307
:107F0000020202021F0200F84848484888000008A0
:107F100010101010080700E03098888888100007BB
:107F200009101010190F0008080808C838180000B8
:107F3000100C030000000070888888888870000F8B
:107F400019101010190F00F09808080890E00008A8
:107F5000111111190C07000000C0C0000000000042
:107F6000001818000000000000C0C0000000000061
:107F700040381800000000008080C0404020000110
:107F80000202060404080040404040404040000215
:107F900002020202020200204040C080800000086D
:107FA00004040602020100100888C87000000000E6
:107FB000001B0000000000C03018884858F0000F77
:107FC00030204748480F0000C0300830C00000187B
:107FD00007020202071800F8888888888870001F46
:107FE00010101010190F00E0100808080810000702
:107FF00008101010100800F80808080810E0001F0A
:1080000010101010080700F8888888888888001FDA
:1080100010101010101000F8888888888888001FB9
:1080200000000000000000E0100808080810000729
:1080300008101010110F00F88080808080F8001F59
:1080400000000000001F00000808F80808000000F9
:1080500010101F101000000000080808F8000008A9
:10806000101010180F0000F880C020100800001F2A
:1080700000000306081000F8000000000000001FC8
:1080800010101010101000F818E000E018F8001F91
:1080900000000100001F00F81860800000F8001FB9
:1080A00000000106181F00E01008080810E0000793
:1080B00008101010080700F80808080898F0001FBA
:1080C00001010101010000E01008080810E00007AC
:1080D00008101030780700F80808080898F0001F0A
:1080E00001010101020C00709088080808100008C6
:1080F00010101111190E00080808F80808080000EF
:1081000000001F00000000F80000000000F8000F51
:1081100018101010180F0018E0000000E018000000
:10812000010E100E0100788000C0C00080780003AE
:108130001C03031C0300000810608060100800107E
:108140000C0300030C10000830C080C03008000091
:1081500000001F00000000080808884838180018B0
:108160001C1211101010000000FC0404000000009C
:10817000003F202000000008708000000000000088
:1081800000010638400000000404FC00000000006C
:1081900020203F00000000406010081060400000F8
:1081A00000000000000000000000000000008080CF
:1081B00080808080808000000206080000000000AF
:1081C000000000000000000040202020C000000E41
:1081D000111111091F0000FC602020608000001FA9
:1081E00008101018070000804020202040000007E1
:1081F000081010100800008060202060FC000007BC
:10820000181010081F00008060202060C0000007C8
:10821000091111110900002020F824242400000075
:10822000001F00000000008060202040E0000007E8
:10823000589090887F0000FC40202020C000001F44
:10824000000000001F0000002020EC0000000010D3
:1082500010101F10101000002020EC000000008003
:1082600080807F00000000FC008040200000001F94
:10827000010106081000040404FC000000000000D6
:10828000000F1010100000E02020E02020C0001F90
:1082900000001F00001F00E040202020C000001F41
:1082A000000000001F0000C060202060C000000F20
:1082B000181010180F0000E040202060800000FF20
:1082C000181010180700008060202040E000000710
:1082D00018101008FF000000E0602020400000009F
:1082E0001F000000000000C02020202040000009E6
:1082F000111112120E00002020F820202000000092
:10830000000F1010100000E000000000E000000F5F
:10831000101010081F000060800000806000000046
:10832000031C1C030000E0000080800000E0000748
:108330001807071807000020408080402000001028
:108340000C03030C10000020C0000080600000003F
:1083500081C63C0300000020202020A060000018FF
:108360001412111010000000C0300830C0000018B6
:1083700007020202071800F8888888888808001F0A
:1083800010101010190F00F8888888888870001F56
:1083900010101010190F00F8080808080808001F2E
:1083A00000000000000000E010080808F800701F3E
:1083B000101010101F7000F8888888888888001FA7
:1083C000101010101010001870C0F8C07018001CA9
:1083D00003001F00031C001008888888483000082C
:1083E00010101010190E00F80000806018F8001F1F
:1083F0001C060100001F00F80102826118F8001F2E
:108400001C060100001F00F880C020100800001F9B
:108410000000030608100000F808080808F8101803
:108420000F000000001F00F818E000E018F8001F1F
:1084300000000100001F00F88080808080F8001F8D
:1084400000000000001F00E01008080810E000070E
:1084500008101010080700F80808080808F8001F9E
:1084600000000000001F00F80808080898F0001F2E
:1084700001010101010000E01008080808100007D0
:1084800008101010100800080808F8080808000074
:1084900000001F000000000830C0008070080000CD
:1084A00010100F03000000E03010F81030E000035F
:1084B0000C081F080C0700081060806010080010EE
:1084C0000C0300030C1000F800000000F800001F6F
:1084D000101010101F7000F80000000000F80000DD
:1084E00001010101011F00F80000F80000F8001F61
:1084F00010101F10101FF80000F80000F8001F10E7
:10850000101F10101F700808F840404080800000C5
:108510001F101010180FF8404040800000F81F1086
:1085200010100807001F00F8808080808000001F66
:1085300010101010190F00108888888890E000082B
:10854000101010100C0700F880F0180818F0001F29
:10855000000F1810180F0000F098080808F8001015
:1085600008070101011F000040202020C000000E6C
:10857000111111091F0000F078282464C000000FB9
:10858000181010180F0000E020202020C000001F4D
:10859000111111110E000000E02020202000000029
:1085A0001F00000000000000E0202020E00000701C
:1085B0001F1010101F7000C020202020C0000007D6
:1085C0000911111109000020E080E080E02000186E
:1085D00006031F030618004020202020C0000008CA
:1085E000101111110E0000E0000000C0E000001F9B
:1085F000080601001F0000E0040808C4E000001F96
:10860000080601001F0000E0008040200000001F5D
:108610000101060810000000E0202020E0001010FA
:108620000F0000001F0000E0C0000000C0E0001FBD
:1086300000030403001F00E000000000E000001F32
:10864000010101011F0000C060202060C000000F78
:10865000181010180F0000E020202020E000001F5C
:10866000000000001F0000E040202060800000FFAC
:10867000181010180700008040202020400000073C
:1086800008101010080000002020E020200000004A
:1086900000001F0000000020C000008060000000FB
:1086A00081C63C03000000C06020FC2060C0000FB9
:1086B0001810FF10180F002040808040200000108C
:1086C0000C03030C100000E000000000E000001F9D
:1086D000101010101F7000E000000000E00000010A
:1086E000020202021F0000E00000E00000E0001FA4
:1086F00010101F10101F00E00000E00000E0001F3D
:1087000010101F10107F2020E0000000000000006B
:108710001F111111110E00E00000000000E0001F09
:108720001111110E001F00E0000000000000001FEA
:10873000111111110E00004020202040800000087F
:1087400011111109070000E000C0602060C0001F87
:10875000020F1810180F00C0202020E000000011A8
:108760000E02021F000000008887000800000020A1
:10877000A8000000C401000830880008A8000020FC
:1087800028530000E0010008000000000000000085
:1087900000000000000000000000000000000000D9
:1087A00000000000000000000000000000000000C9
:1087B00000000000000000000000000000000000B9
:1087C00000000000000000000000000000000000A9
:1087D0000000000000000000000000000000000099
:1087E0000000000000000000000000000000000089
:1087F0000102030401020304060708090100020044
:108800000400060008000A000C00100020004000D0
:1088100080000001000000000000000000A24A04E7
:108820000000000000000000010203040607080920
:040000050800018965
:00000001FF
